:100000000C9411020C942C020C942C020C942C02D3
:100010000C942C020C942C020C942C020C942C02A8
:100020000C942C020C94270C0C942C020C942C0293
:100030000C9409160C942C020C942C020C942C0297
:100040000C942C020C942C020C94200B0C942C027B
:100050000C948E040C942C020C9458040C942C02D6
:100060000C942C0D0C942C020C9433150C942C0233
:100070000A0D466C69676874436F6E74726F6C0A20
:100080000D48617264776172653A25642E25640AB1
:100090000D536F6674776172653A5625642E256438
:1000A000256320000A0D3D3D3D3D3D3D3D3D3D3D2F
:1000B0003D3D3D3D3D3D3D3D3D3D3D3D3D3D3D3D70
:1000C0003D3D3D3D000A0D496E69742E2045455069
:1000D000524F4D3A2047656E6572696572652044DE
:1000E000656661756C742D506172616D65746572C1
:1000F0002E2E2E000A0D414343206E696368742042
:1001000061626765676C696368656E21000A0D420C
:10011000656E75747A6520506172616D6574657283
:100120007361747A202564000A0D4162676C656909
:100130006368204C756674647275636B73656E7367
:100140006F722E2E004F4B0A0D000A0D5374657509
:100150006572756E673A200048656164696E67482C
:100160006F6C64004E65757472616C000A0A0D0054
:100170002E005B25695D002B2B204D696B726F4B48
:100180006F70746572202B2B0048573A5625642EE9
:1001900025642053573A25642E2564256300536552
:1001A0007474696E673A202564200028632920480A
:1001B0006F6C676572204275737300486F65686580
:1001C0003A202020202025356900536F6C6C486F41
:1001D0006568653A20253569004C756674647275EA
:1001E000636B3A20253569004F6666202020202069
:1001F000203A20253569004B65696E65200048F678
:1002000068656E726567656C756E6700616B742EEC
:10021000204C616765004E69636B3A2020202020E6
:100220002025356900526F6C6C3A20202020202058
:10023000253569004B6F6D706173733A202020255E
:100240003569004B313A25346920204B323A253448
:100250006920004B333A25346920204B343A253449
:100260006920004B353A25346920204B363A253435
:100270006920004B373A25346920204B383A253421
:100280006920004E693A2534692020526F3A25349E
:1002900069200047733A253469202047693A25349C
:1002A00069200050313A253469202050323A2534F3
:1002B00069200050333A253469202050343A2534DF
:1002C0006920004779726F202D2053656E736F721D
:1002D000004E69636B202534692028253369290085
:1002E000526F6C6C2025346920282533692900471A
:1002F00069657220253469202825336929004E69F3
:10030000636B2025346920282533692900526F6CDE
:100310006C202534692028253369290047696572D6
:100320002025346920282533692900414343202DA5
:100330002053656E736F72004E69636B20253469BC
:1003400020282533692900526F6C6C2025346920E0
:10035000282533692900486F6368202534692028DF
:1003600025336929005370616E6E756E673A2020DF
:1003700025356900456D70662E506567656C3A25B8
:100380003569004B6F6D7061737320202020202031
:1003900020005269636874756E673A2020253569BC
:1003A000004D657373776572743A202025356900B6
:1003B00053746172743A2020202020253569005042
:1003C0006F7469313A202025336900506F746932A7
:1003D0003A202025336900506F7469333A20202574
:1003E000336900506F7469343A2020253369005313
:1003F0006572766F202000536574706F696E74208B
:1004000020253369005374656C6C756E673A20253E
:1004100033690052616E67653A2533692D2533696A
:10042000000011241FBECFEFD0E1DEBFCDBF13E02F
:10043000A0E0B1E0E2EEF9E702C005900D92A23A29
:10044000B107D9F717E0A2EAB3E001C01D92A43BBF
:10045000B107E1F70C9467020C940000FB018630B1
:1004600008F085E0489FD0011124AC59BF4F842F7C
:100470009927019724F00E94DD3C0192FACF08955C
:10048000282FFB01863008F025E0429FD00111247F
:10049000AC59BF4F842F9927019724F001900E94F7
:1004A000E53CFACFA2E0B0E0022E0E94E53C0895C0
:1004B000A2E0B0E09D010E94DD3C802D863028F056
:1004C00082E0D901082E0E94E53C99270895CFEFDC
:1004D000D0E1DEBFCDBF14B815B897EEE92E93E09A
:1004E000F92E8EEC9FEFE80EF91EF7FEFACF88EE9C
:1004F000E82E83E0F82E189B02C08BE001C08AE052
:100500008093000181E887B98FEF88B98BE184B9C6
:1005100081E085B98EE38AB9579A87EF8BB984B7A2
:10052000877F84BF80916000886180936000109213
:10053000600080ED97E09093C0038093BF0310921A
:100540001304109212041092100710920F071092C9
:10055000150410921404109217041092160480913E
:1005600000018A3011F4289801C0289A0E94D70B04
:100570000E948E070E94F4150E94DE0C0E94FC145B
:10058000789410920E0683E480930F0687E08093A0
:10059000100686E690E09F938F9383E490E09F930C
:1005A0008F931F921F92809100016AE00E946D3C20
:1005B000892F99279F938F93809100010E946D3C12
:1005C00099279F938F9380E790E09F938F931F923B
:1005D0000E9496088DB79EB70D960FB6F8949EBFF1
:1005E0000FBE8DBF84EA90E09F938F931F920E946D
:1005F0009608299A0F900F900F9001E010E0D80113
:100600000E94DD3C802D843461F185EC90E09F9365
:100610008F931F920E9496080E94BE16C0E00F9012
:100620000F900F90C23039F0C33019F40E94E117D7
:1006300004C0C43010F00E944F1747E467E377E02E
:100640008C2F0E944002CF5FC63060F3A2E0B0E082
:1006500083E0082E0E94E53C84E4D801082E0E9425
:10066000E53CA4E0B0E00E94DD3C802D853050F0F8
:1006700084EF90E09F938F931F920E9496080F90B3
:100680000F900F900E94580247E467E377E00E94C2
:100690002E020E94580299279F938F938DE091E03C
:1006A0009F938F931F920E94960880913F070F900F
:1006B0000F900F900F900F9080FF20C088E291E084
:1006C0009F938F931F920E94960888EE93E00E945A
:1006D000CE0B7C010E94E40C0F900F900F90C7018D
:1006E0000E94FD0B8823D9F385E491E09F938F93BB
:1006F0001F920E9496080F900F900F900E94E11990
:10070000809100018A3011F4289801C0289A80ED68
:1007100097E09093C0038093BF0388EE93E090939B
:1007200009068093080685E5809303068AE491E034
:100730009F938F931F920E94960880913F070F907E
:100740000F900F9082FF03C088E591E002C084E61D
:1007500091E09F938F931F920E9496080F900F90A5
:100760000F908CE691E09F938F931F920E949608C2
:100770000E94041088E893E1909387038093860396
:100780000F900F900F908091C303882309F462C0EB
:100790001092C3030E94BC240E948D21209100016D
:1007A0002A3011F4289801C0289A809101038823E7
:1007B00021F081508093010310C08093A2038093A5
:1007C000A3031092F8031092F7031092F60310920D
:1007D000F5031092F4031092F30380911804882318
:1007E00029F0809118048150809318048091860329
:1007F00090918703892B01F585E090E09093870322
:10080000809386030E94161580910403909105033E
:100810008F5F9F4FF9F4809111048823D9F080E114
:1008200097E29093C0038093BF0380E890E0909399
:100830000503809304030EC0809186039091870383
:10084000019790938703809386032A3011F42898A8
:1008500001C0289A0E94AC070E947806C7010E9436
:10086000FD0B882309F48FCF80914F07282F332762
:1008700080910E0390910F03821793079CF480914F
:100880000403909105038F5F9F4F61F480E797E128
:100890009093C0038093BF0380E093E0909305039F
:1008A0008093040384E690E00E94CE0B7C016BCF22
:1008B0001F920F920FB60F9211248F939F93EF9375
:1008C000FF93809103038823E1F48091B503909115
:1008D000B60301969093B6038093B503FC01EB52E7
:1008E000FB4FE081ED3019F08639910539F4109213
:1008F000B6031092B50381E080930303E093C60032
:1009000004C01092B6031092B503FF91EF919F912E
:100910008F910F900FBE0F901F9018951F920F92FE
:100920000FB60F9211242F933F934F935F938F93A2
:100930009F93AF93BF93EF93FF9390E08091C60096
:100940008093B0035091BB03563910F09093BC03D1
:100950008091B0038D3009F05FC08091BC0382307C
:1009600009F05AC09093BC03852F9927885E994F50
:10097000FC01329740812091B7033091B803241BCA
:100980003109DC0111978C91281B3109C9019F7035
:100990009093B8038093B70346E0969587954A9560
:1009A000E1F7982F935C9093B9032F733070235C19
:1009B0002093BA038081981729F48C91281711F499
:1009C00091E006C090E08091AD038F5F8093AD030E
:1009D0008091AF03882309F06EC0992309F46BC09E
:1009E00081E08093AF035093AC03E52FFF27E85ECF
:1009F000F94F8DE0808380911A06823509F05BC043
:100A000088E190E02CE00FB6F894A8958093600000
:100A10000FBE209360004FC02091BC03822F992706
:100A200081309105F9F0823091051CF4892B21F079
:100A300040C0029711F13DC08091B003833239F478
:100A40008091AF03882319F481E08093BC038091E7
:100A5000B0038093180681E08093BB038091B003BC
:100A6000992722C02F5F2093BC03E52FFF27E85E64
:100A7000F94F8091B003808309C0E52FFF27E85E1E
:100A8000F94F8091B0038083563920F45F5F509313
:100A9000BB0302C01092BC032091B0038091B70346
:100AA0009091B803820F911D9093B8038093B70380
:100AB00002C01092BC03FF91EF91BF91AF919F9143
:100AC0008F915F914F913F912F910F900FBE0F909B
:100AD0001F901895AC01A0E0B0E09D01A817B907E0
:100AE00048F4E5EDF4E08191280F311D1196A4172B
:100AF000B507C8F33F70FD01EB52FB4FC90156E04B
:100B0000969587955A95E1F7835C80831196FD0150
:100B1000EB52FB4F2F733070822F835C8083AA527D
:100B2000BB4F8DE08C93109203038091D50480938A
:100B3000C60008951F93CF93DF93382FEA01722FD9
:100B400010E083E28093D5046093D6043093D704F9
:100B5000A3E0B0E0772309F458C0772311F4972F6E
:100B600007C0FE01E10FF11D1F5F9081715011F46C
:100B7000472F0EC0FE01E10FF11D1F5F4081715034
:100B800039F0FE01E10FF11D1F5F6081715001C05E
:100B9000672FFD01EB52FB4F892F86958695835C6D
:100BA00080831196FD01EB52FB4F892F99278370AB
:100BB000907024E0880F991F2A95E1F755279A0134
:100BC00094E0369527959A95E1F7822B835C808394
:100BD0001196FD01EB52FB4F4F705070440F551FA3
:100BE000440F551F862F992726E0969587952A95BD
:100BF000E1F7842B835C80831196FD01EB52FB4F60
:100C00006F73635C60831196A5CFCD010E946A0566
:100C1000DF91CF911F9108951F93CF93DF93EC0144
:100C200010E0662309F460C0A22FBB271297E42FBF
:100C3000FF27E85EF94F30813D534F5FE42FFF27D8
:100C4000E85EF94F50815D534F5FE42FFF27E85E68
:100C5000F94F70817D534F5FE42FFF27E85EF94F16
:100C6000E081ED534F5F842F9927A817B907E4F16E
:100C7000832F9927880F991F880F991F352F329539
:100C80003F70382B852F99278F709070F4E0880F74
:100C9000991FFA95E1F7572F56955695582B872FA0
:100CA00099278370907076E0880F991F7A95E1F705
:100CB0008E2B61506F3FC1F0FE01E10FF11D3083BB
:100CC0001F5F61506F3F81F0FE01E10FF11D508306
:100CD0001F5F61506F3F41F0FE01E10FF11D808306
:100CE0001F5F662309F0A3CFDF91CF911F91089575
:100CF000CF93DF93CDB7DEB722970FB6F894DEBF60
:100D00000FBECDBF8091AF03882309F4ECC08FEFF5
:100D10008093010380911A0699278B36910509F477
:100D200067C08C36910594F48336910561F1843661
:100D3000910524F481369105D1F0D3C08736910511
:100D400009F463C08836910589F1CBC081379105DC
:100D500009F45FC0813791050CF47DC0843791059B
:100D600009F43FC08637910509F44BC0BAC0209101
:100D7000AC0343E062E0CE0101960E940C0689813B
:100D800080930203AEC02091AC0343E06BE083E0AC
:100D900096E00E940C068091E70390910506892B4E
:100DA0008093E70381E08093B2039BC02091AC0362
:100DB00043E062E0CE0101960E940C068091E703B9
:100DC0009981892B8093E7038A818F3F21F481E009
:100DD0008093A90302C01092A90381E08093B3031A
:100DE00080C02091AC0343E064E085EA93E006C054
:100DF0002091AC0343E0642F82EA93E00E940C064A
:100E000070C081E08093B1036CC081E08093B40333
:100E100068C02091AC0343E062E0CE0101960E94DD
:100E20000C0689818F3F61F0863010F085E0898360
:100E300047E467E377E089810E942E02898102C03E
:100E40000E94580227E447E357E06091D404855B91
:100E50000E949A0546C02091AC0343E067E487E313
:100E600097E00E940C0680911A0647E467E377E05A
:100E70008B560E944002A2E0B0E080911A068B5689
:100E8000082E0E94E53C809162079927AA27BB277C
:100E9000BC01CD0124EC39E040E050E00E944E3C22
:100EA000DC01CB018093820390938303A09384039E
:100EB000B0938503809163079927AA27BB27BC01BC
:100EC000CD010E944E3CDC01CB0180937E039093C8
:100ED0007F03A0938003B09381030E9458020E9475
:100EE00071181092AF0322960FB6F894DEBF0FBEB2
:100EF000CDBFDF91CF910895CF93C82F8A3019F4D9
:100F00008DE00E947C078091C00085FFFCCFC093DC
:100F1000C60080E090E0CF910895089588E1809325
:100F2000C1008091C00082608093C0008091C100A8
:100F300080688093C1008091C10080648093C1006B
:100F40008AE28093C40088EC90E00E94CE0B9093DC
:100F5000020680930106089580910303882309F413
:100F60008AC08091B403882371F0809103038823A1
:100F700051F02BE043E056E06091D40487E40E94F6
:100F80009A051092B40380910106909102060E9486
:100F9000FD0B882321F48091B2038823B1F0809166
:100FA0000303882391F022E44EEA56E06091D404D2
:100FB00084E40E949A051092B20384EF91E00E94AB
:100FC000CE0B9093020680930106609102036F3F5F
:100FD00091F0862F992734E0880F991F3A95E1F711
:100FE0008F5F9E4F605D20E1AC0181E40E949A0515
:100FF0008FEF809302038091B303882351F1809196
:101000000303882331F10E940D101092B303309135
:10101000AA03832F8F5F8093AA03843021F060910D
:10102000A903662359F026E14BE057E060E084E332
:101030000E949A058FEF8093AA030BC024E1829F40
:10104000C0011124805F9C4FAC01832F8F5C0E94F4
:101050009A058091B103882371F08091030388235E
:1010600051F02AE04EE056E06091D40486E50E94FB
:101070009A051092B1030895982F8091F00681305F
:1010800069F48091E803E82FFF27E05FFC4F90832D
:101090008F5F8093E80321E030E005C0892F0E9434
:1010A0007C07282F3327C90108950F931F93CF93EF
:1010B000DF938C01EB01672B39F0F80181918F01EF
:1010C0000E943C082197C9F7DF91CF911F910F91A2
:1010D00008950F931F93CF93DF938C01EB01672B40
:1010E00041F0F8010F5F1F4F84910E943C08219747
:1010F000C1F7DF91CF911F910F910895CF93C82F22
:10110000181634F480E20E943C08C1501C16D4F337
:10111000CF910895CF93C82F181634F480E30E941E
:101120003C08C1501C16D4F3CF9108952F923F92E2
:101130004F925F926F927F928F929F92AF92BF92E7
:10114000CF92DF92EF92FF920F931F93CF93DF9393
:10115000CDB7DEB7E0970FB6F894DEBF0FBECDBFB8
:1011600026968FAD26972896EEADFFAD28971CA644
:101170001DA61EA61FA68093F006A8E46A2E712C59
:101180006C0E7D1E5F01C50105C0053239F0089463
:10119000A11CB11CF50104910023B9F7B501681B2E
:1011A000790B11F00E946908002309F430C20894F9
:1011B000A11CB11C552458AA252C1FEF59A6F501D6
:1011C0000894A11CB11C0491053721F0802F806286
:1011D0008837F1F450FE0EC0F30124E030E0620ED7
:1011E000731E80819181A281B3818CA79DA7AEA738
:1011F000BFA70EC0F301A2E0B0E06A0E7B1E8081A3
:1012000091819C01442755272CA73DA74EA75FA796
:10121000003221F489A5882391F61BC0033211F412
:1012200038E081C00A3211F00D3289F40A3251F4EB
:10123000F30142E050E0640E751E208022200CF085
:10124000BECF219450E1552A8FED5822B8CF0B32F2
:1012500011F409A7B4CF0E32C1F5F5010894A11C11
:10126000B11C04910A3279F4F301A2E0B0E06A0EF5
:101270007B1E60817181BFEF6F3F7B0714F46FEFBE
:101280007FEF162F9CCF60E070E0802F80538A3074
:10129000A0F4CB01F3E0880F991FFA95E1F7860FD0
:1012A000971F680F791F600F711D60537040F50123
:1012B0000894A11CB11C0491E8CFEFEF6F3F7E07AB
:1012C00014F46FEF7FEF162F7FCF003329F454FC17
:1012D00076CFF0E25F2A73CF802F81538930D8F424
:1012E00060E070E0CB01E3E0880F991FEA95E1F739
:1012F000860F971F680F791F600F711D6053704034
:10130000F5010894A11CB11C0491802F80538A30F0
:1013100048F3262E59CF083619F424E0522A4FCF2D
:101320000C3619F431E0532A4ACF033661F44E01EA
:101330000894811C911CF30142E050E0640E751E7C
:10134000808189831BC1043421F0043611F00936F1
:10135000B1F5043411F451E0552A50FE0AC0F301EE
:1013600084E090E0680E791E2081318142815381B2
:101370000CC0F30142E050E0640E751E8081918143
:101380009C01442737FD4095542F2CA73DA74EA71D
:101390005FA78CA59DA5AEA5BFA5B7FF0DC0B09555
:1013A000A095909581959F4FAF4FBF4F8CA79DA75C
:1013B000AEA7BFA78DE289A77AE0472E7BC00F3486
:1013C00011F00F3639F40F3411F491E0592A68E026
:1013D000462E6FC00037A1F4F301A2E0B0E06A0E20
:1013E0007B1E808191819C01442755272CA73DA716
:1013F0004EA75FA750E1452E30E4532A08E759C0B5
:101400000337C1F5F30142E050E0640E751E8080A1
:1014100091808114910489F44E010894811C911CDF
:1014200088E289838EE6F401818385E78B838CE6ED
:101430008C838D8389E28E831F8217FD13C0812FD9
:10144000992787FD9095AC0160E070E0C4010E948F
:10145000D93A009729F0D82ED8181D150CF090C055
:10146000D12E8EC0F40101900020E9F73197DE2ED5
:10147000D81886C0053511F0053739F4053511F453
:10148000F1E05F2A4AE0442E14C0083519F008370D
:1014900009F06CC030E1432E53FE0BC02CA53DA5D6
:1014A0004EA55FA5211531054105510511F030E428
:1014B000532A19A618AB17FD02C04FED542229E29A
:1014C000822E912C8C0E9D1E8CA59DA5AEA5BFA530
:1014D0000097A105B10521F498A9992309F43FC00B
:1014E000C42CDD24EE24FF2433242CA53DA54EA5D9
:1014F0005FA52C153D054E055F0510F091E0392ED6
:101500006CA57DA58EA59FA5A70196010E94A03C74
:10151000DC01CB01182F8A3010F4105D04C0195A79
:10152000083509F41F7DD4011E934D016CA57DA5DE
:101530008EA59FA5A70196010E94A03C2CA73DA7C0
:101540004EA75FA7332081F6B8E04B1641F453FE57
:1015500006C0103321F080E3F40182934F01CE01E5
:101560000196D82ED818F8E2DF0E0BC0002309F43C
:101570004EC04E010894811C911C098381E0D82E35
:1015800019A61D2DC8A8CD18C7FCCC2489A5882371
:1015900011F01F5F02C056FC1E5F1C0DE52CFF24DE
:1015A000C70180739070892B21F4822D811B0E94CA
:1015B0007E0889A5882329F061E070E0CE01899634
:1015C00009C0E6FE09C080E38AA70BA762E070E0CD
:1015D000CE018A960E945508C7018073907080974B
:1015E00021F4822D811B0E948A088C2D0E948A087A
:1015F0008D2D992787FD9095BC01C4010E94550847
:10160000E4FEC1CD822D811B0E947E08BCCDE096F8
:101610000FB6F894DEBF0FBECDBFDF91CF911F9103
:101620000F91FF90EF90DF90CF90BF90AF909F9081
:101630008F907F906F905F904F903F902F90089584
:101640001F920F920FB60F9211242F933F935F9327
:101650006F937F938F939F93AF93BF938091C603B4
:1016600081508093C6038F3FB9F489E08093C6030D
:10167000809106038F5F817080930603882319F49D
:1016800081E08093C3038091C4039091C5030196C8
:101690009093C5038093C4038091BF039091C003CE
:1016A0000297C8F08091BF039091C0030197909377
:1016B000C0038093BF038091BF039091C00320912A
:1016C00004033091050382239323892B11F021E039
:1016D00009C020E007C020E08FEF9FEF9093050343
:1016E0008093040380910001222331F08A3011F4A9
:1016F0005A9A07C0479A05C08A3011F45A9801C017
:10170000479880913F0783FF3BC0349B0AC080917C
:10171000C1039091C20301969093C2038093C103C9
:101720002FC08091C1039091C203892B79F08091E1
:10173000C1039091C203805A9F4040F48091C1033D
:101740009091C203909328048093270480912704EA
:10175000909128042091250430912604821B930B3C
:10176000845E9D4F68E671E00E948D3C845B9040F2
:1017700090932404809323041092C2031092C10317
:10178000BF91AF919F918F917F916F915F913F91A9
:101790002F910F900FBE0F901F9018952091C403AA
:1017A0003091C503280F391FC901019608958AE0B9
:1017B00090E00E94CE0B9093C8038093C70382E011
:1017C00085BD83EA84BD17BC88E788BD96E096BDD9
:1017D00083EC8093B0009093B100809170008260A0
:1017E0008093700080916E00816080936E008AE02B
:1017F0008093B3001092B20008952091C4033091F9
:10180000C503821B930B892F99278695807490704E
:101810000895CF93DF930E94CE0BEC01CE010E947E
:10182000FD0B8823D9F3DF91CF910895CF93DF93F8
:101830000E94CE0BEC0103C08FEE80937A00CE01A4
:101840000E94FD0B8823C1F3DF91CF9108951F9271
:101850000F920FB60F9211242F933F934F935F93E4
:101860006F937F938F939F93AF93BF93CF93DF93A8
:10187000EF93FF93809107038150809307038F3F7D
:1018800009F085C083E88093B00080917003C82F71
:10189000DD27D093BE03C093BD0380916C07609198
:1018A000590780FF2AC0772788279927209161044C
:1018B00030916204409163045091640457FF04C066
:1018C00021583F4F4F4F5F4FA7E0559547953795AC
:1018D0002795AA95D1F70E944E3C97FF04C061500E
:1018E0007E4F8F4F9F4FF9E0959587957795679538
:1018F000FA95D1F7C60FD71F29C0772788279927D0
:101900002091610430916204409163045091640419
:1019100057FF04C021583F4F4F4F5F4FE7E05595A9
:10192000479537952795EA95D1F70E944E3C97FF4A
:1019300004C061507E4F8F4F9F4F39E0959587953A
:10194000779567953A95D1F7C61BD70BD093BE0311
:10195000C093BD0380915A0799272091BD03309110
:10196000BE032817390734F080915B079927821747
:10197000930724F49093BE038093BD038091BD032D
:101980008093B30080915C078093070304C083E0D9
:101990008093B0005F98FF91EF91DF91CF91BF915D
:1019A000AF919F918F917F916F915F914F913F91F7
:1019B0002F910F900FBE0F901F90189510927C00E2
:1019C0008FEE80937A0008950F931F93CF93DF9348
:1019D00003E010E0D8010E94DD3C802DC82FDD27F8
:1019E000C531D10508F02A97C7BD84E690E00E9472
:1019F000160C80910803909109038255934010F4CE
:101A0000C0E0D0E0CA3FD105C0F4C7BD82E390E09A
:101A10000E94160C80E791E09F938F931F920E9483
:101A2000960880910803909109030F900F900F90F2
:101A30008458934010F02196E5CFD8010C2E0E94D7
:101A4000E53CC093FE068CE291E00E94160CDF910B
:101A5000CF911F910F9108951F920F920FB60F9281
:101A60001124EF92FF920F931F932F933F934F9365
:101A70005F936F937F938F939F93AF93BF93CF9316
:101A8000DF93EF93FF9310927A008091E003682F29
:101A900077278F5F8093E0036530710509F48EC06E
:101AA00066307105BCF46230710509F44AC06330D8
:101AB00071053CF46115710531F161307105C1F1B9
:101AC0007DC26330710509F446C06430710509F4C4
:101AD0005DC074C26830710509F4C3C06930710516
:101AE0004CF46630710509F482C06730710509F461
:101AF0009BC064C26930710509F4D0C06A307105B9
:101B000009F4DCC15BC280917800909179009093D8
:101B1000E2038093E10381E08093DF038091C903B6
:101B20009091CA0301969093CA038093C9034AC255
:101B300080917800909179009093E4038093E3037F
:101B40008EC080917800909179009093E603809305
:101B5000E50384E0B0C180910E0390910F039C01D6
:101B6000220F331F280F391F809178009091790040
:101B70000E94793C260F371F369527953695279575
:101B800030930F0320930E0386E095C180916B0480
:101B900090916C042091780030917900821B930B16
:101BA0009093F2068093F1068091F1069091F206EF
:101BB0009093D8038093D70387E07DC1809178000C
:101BC0009091790020916D0430916E04821B930BEB
:101BD0009093FD068093FC068091FC069091FD0693
:101BE0009093D6038093D5031092DF03EBC18091CD
:101BF00000012091E1033091E2038A3049F48091A1
:101C0000780090917900820F931F9695879506C072
:101C10008091780090917900820F931F9093DA035E
:101C20008093D90381E047C1809100012091E303B3
:101C30003091E4038A3049F48091780090917900E2
:101C4000820F931F9695879506C08091780090919A
:101C50007900820F931F9093DC038093DB0382E073
:101C60002AC1809100012091E5033091E6038A307A
:101C700049F48091780090917900820F931F969596
:101C8000879506C08091780090917900820F931F0C
:101C90009093DE038093DD0385E00DC18091780091
:101CA00090917900AA2797FDA095BA2FBC01CD018C
:101CB0000E948C3B7B018C018091670490916804A9
:101CC000A0916904B0916A049C01AD01C801B701FB
:101CD0000E94E63ADC01CB01BC01CD010E946F3BC2
:101CE000DC01CB019093D4038093D3038091F10660
:101CF0009091F2068091F1069091F20697FF03C051
:101D0000909581959F4F97FD0396AC01559547950A
:101D1000559547958091FC069091FD068091FC06B3
:101D20009091FD0697FF03C0909581959F4F9C0170
:101D300097FF02C02D5F3F4F359527953595279525
:101D4000240F351F8091D3039091D403820F931FEA
:101D50009093D4038093D3038091D3039091D403C1
:101D6000029724F18091670490916804A09169041E
:101D7000B0916A0420E030E048E454E4BC01CD01B5
:101D80000E94963B88230CF044C080916704909198
:101D90006804A0916904B0916A042AE037ED43EA2F
:101DA0005CE3BC01CD010E94E73A29C08091D303D6
:101DB0009091D4038F5F9F4F64F580916704909159
:101DC0006804A0916904B0916A0420E030E046E123
:101DD00054E4BC01CD010E94993B1816D4F48091C3
:101DE000670490916804A0916904B0916A042AE0A4
:101DF00037ED43EA5CE3BC01CD010E94E63ADC0129
:101E0000CB018093670490936804A0936904B09316
:101E10006A0481E08093CD038091780090917900ED
:101E20009093F4068093F3068091D3039091D403AA
:101E30009C01442737FD4095542F809129049091AF
:101E40002A04A0912B04B0912C04820F931FA41F8D
:101E5000B51F8093290490932A04A0932B04B09378
:101E60002C042091290430912A0440912B04509194
:101E70002C0457FF04C021503C4F4F4F5F4F7AE076
:101E800055954795379527957A95D1F780912904EF
:101E900090912A04A0912B04B0912C04821B930BE7
:101EA000A40BB50B8093290490932A04A0932B04D0
:101EB000B0932C0483E08093DF0384C080910107FA
:101EC000909102072091780030917900820F931F42
:101ED00090930207809301078091F9068F5F8093AA
:101EE000F9068091F906853008F468C08091780081
:101EF0009091790090930903809308031092F9065A
:101F00008091F5069091F606209101073091020725
:101F1000821B930B20910F0430911004821B930BB2
:101F20009093CC038093CB0380910107909102079B
:101F3000EC01EE27D7FDE095FE2F20910A033091AA
:101F40000B0340910C0350910D03DA01C901880F76
:101F5000991FAA1FBB1F820F931FA41FB51FC80F75
:101F6000D91FEA1FFB1FF7FF03C02396E11DF11DD8
:101F700082E0F595E795D795C7958A95D1F7C093F7
:101F80000A03D0930B03E0930C03F0930D038091AD
:101F90000A0390910B03A0910C03B0910D039C01D7
:101FA0008091F5069091F606821B930B9093100496
:101FB00080930F0410920207109201071092DF0322
:101FC0001092E0038091DF0380937C008091E00316
:101FD000882319F08FEE80937A00FF91EF91DF91C3
:101FE000CF91BF91AF919F918F917F916F915F91B1
:101FF0004F913F912F911F910F91FF90EF900F9074
:102000000FBE0F901F90189590E2E0E1F3E08FE48F
:102010009193815087FFFCCF08951F93CF93DF9357
:102020008091E70380FF0FC08091EB03882311F0BC
:10203000815002C080916A038093EB030E940410D8
:102040008FEF8093AA038091E70381FF0AC08091FC
:10205000EB038F5F8093EB030E9404108FEF80935C
:10206000AA038091E703992780FF04C081FF02C083
:102070001092EB0381E18093E8038091EB039927B1
:102080009F938F9382E791E09F938F9311E01F932B
:102090000E9496080F900F900F900F900F908091D4
:1020A000EB03C82FDD27C530D10509F45DC2C6306A
:1020B000D105ACF4C230D10509F4E2C0C330D1057A
:1020C00034F4209719F1219709F472C08AC4C330FF
:1020D000D10509F443C1249709F4ABC182C4C830C7
:1020E000D10509F496C3C930D10544F4C630D105F1
:1020F00009F40BC3279709F46CC373C4C930D10525
:1021000009F4C9C32A9709F41AC46BC41092E803EE
:1021100087E791E09F938F931F930E94960884E135
:102120008093E8030F900F900F9086E690E09F93C6
:102130008F9383E490E09F938F93DF93CF9380916D
:1021400000016AE00E946D3C892F99279F938F932D
:10215000809100010E946D3C99279F938F9389E89D
:1021600091E09F938F931F930E94960888E280933B
:10217000E8038DB79EB70D960FB6F8949EBF0FBEBD
:102180008DBF0E94580299279F938F938EE991E00B
:102190009F938F931F930E9496088CE38093E8038C
:1021A0000F900F900F900F900F908BEA91E05FC00F
:1021B00080913F0780FF49C01092E80380910F048F
:1021C000909110049F938F938BEB91E09F938F934B
:1021D0001F930E94960884E18093E8030F900F906C
:1021E0000F900F900F9080910D0490910E049F938B
:1021F0008F938AEC91E09F938F931F930E94960890
:1022000088E28093E8030F900F900F900F900F904B
:1022100080910803909109039F938F9389ED91E03A
:102220009F938F931F930E9496088CE38093E803FB
:102230000F900F900F900F900F908091FE069927AE
:102240009F938F9388EE91E06FC384E18093E803BE
:1022500087EF91E09F938F931F930E94960888E2E7
:102260008093E8030F900F900F908EEF91E09F9373
:102270008F931F930E9496080F900F900F90B6C3F4
:102280001092E8038CE092E09F938F931F930E943B
:10229000960884E18093E8030F900F900F9080914F
:1022A000610490916204A0916304B0916404B7FF4B
:1022B00004C081509C4FAF4FBF4F6AE0B595A795C2
:1022C000979587956A95D1F7BF93AF939F938F9317
:1022D00086E192E09F938F931F930E94960888E275
:1022E0008093E8038DB79EB707960FB6F8949EBF0C
:1022F0000FBE8DBF8091590490915A04A0915B0448
:10230000B0915C04B7FF04C081509C4FAF4FBF4FEA
:102310005AE0B595A795979587955A95D1F7BF93AC
:10232000AF939F938F9385E292E09F938F931F9338
:102330000E9496088CE38093E8038DB79EB70796BA
:102340000FB6F8949EBF0FBE8DBF80912704909169
:1023500028049F938F9384E392E0E6C21092E803EF
:1023600080910F07909110079F938F9380910D0795
:1023700090910E079F938F9383E492E09F938F93A6
:102380001F930E94960884E18093E8038DB79EB75F
:1023900007960FB6F8949EBF0FBE8DBF80911307AE
:1023A000909114079F938F9380911107909112073A
:1023B0009F938F9383E592E09F938F931F930E9447
:1023C000960888E28093E8038DB79EB707960FB60C
:1023D000F8949EBF0FBE8DBF80911707909118078C
:1023E0009F938F9380911507909116079F938F93DA
:1023F00083E692E09F938F931F930E9496088CE34D
:102400008093E8038DB79EB707960FB6F8949EBFEA
:102410000FBE8DBF80911B0790911C079F938F93D8
:102420008091190790911A079F938F9383E792E009
:10243000CAC21092E80380913807E82FFF27EE0FF9
:10244000FF1FE55FF84F808191819F938F9380916B
:102450003707E82FFF27EE0FFF1FE55FF84F80815A
:1024600091819F938F9383E892E09F938F931F9323
:102470000E94960884E18093E8038DB79EB7079683
:102480000FB6F8949EBF0FBE8DBF80913A07E82F1C
:10249000FF27EE0FFF1FE55FF84F808191819F932B
:1024A0008F9380913907E82FFF27EE0FFF1FE55F1D
:1024B000F84F808191819F938F9383E992E09F935E
:1024C0008F931F930E94960888E28093E8038DB74C
:1024D0009EB707960FB6F8949EBF0FBE8DBF809132
:1024E0003C07E82FFF27EE0FFF1FE55FF84F8081C5
:1024F00091819F938F9380913B07E82FFF27EE0FE9
:10250000FF1FE55FF84F808191819F938F9383EA4E
:1025100092E09F938F931F930E9496088CE3809381
:10252000E8038DB79EB707960FB6F8949EBF0FBE0F
:102530008DBF80913E07E82FFF27EE0FFF1FE55F5D
:10254000F84F808191819F938F9380913D07E82F71
:10255000FF27EE0FFF1FE55FF84F808191819F936A
:102560008F9383EB92E02FC21092E80383EC92E00A
:102570009F938F931F930E949608809100010F9064
:102580000F900F908A3009F05AC084E18093E803DD
:1025900080917704909178049F938F938091DD03CD
:1025A0009091DE032091770430917804821B930B85
:1025B0009F938F9381ED92E09F938F931F930E943F
:1025C000960888E28093E8038DB79EB707960FB60A
:1025D000F8949EBF0FBE8DBF8091750490917604D4
:1025E0009F938F938091DB039091DC03209175047E
:1025F00030917604821B930B9F938F9380EE92E031
:102600009F938F931F930E9496088CE38093E80317
:102610008DB79EB707960FB6F8949EBF0FBE8DBFBD
:1026200080917304909174049F938F938091A60777
:102630009091A7079F938F938FEE92E0C4C184E19E
:102640008093E803809177049091780497FD019638
:10265000959587959F938F938091DD039091DE03ED
:102660002091770430917804821B930B9F938F9372
:102670008EEF92E09F938F931F930E94960888E2BB
:102680008093E8038DB79EB707960FB6F8949EBF68
:102690000FBE8DBF809175049091760497FD0196D1
:1026A000959587959F938F938091DB039091DC03A1
:1026B0002091750430917604821B930B9F938F9326
:1026C0008DE093E09F938F931F930E9496088CE375
:1026D0008093E8038DB79EB707960FB6F8949EBF18
:1026E0000FBE8DBF809173049091740497FD019685
:1026F000959587959F938F938091A6079091A707B3
:102700009F938F938CE193E05EC11092E8038BE27C
:1027100093E09F938F931F930E94960884E1809388
:10272000E8030F900F900F9080916D0490916E04CC
:102730009F938F938091D5039091D6039F938F930E
:1027400088E393E09F938F931F930E94960888E2FB
:102750008093E8038DB79EB707960FB6F8949EBF97
:102760000FBE8DBF80916B0490916C049F938F93EB
:102770008091D7039091D8039F938F9387E493E040
:102780009F938F931F930E9496088CE38093E80396
:102790008DB79EB707960FB6F8949EBF0FBE8DBF3C
:1027A0008091670490916804A0916904B0916A04D3
:1027B000BC01CD010E946F3BDC01CB019F938F9345
:1027C00080918E0790918F079F938F9386E593E07A
:1027D000FAC084E18093E80380910E0390910F0387
:1027E0009F938F9385E693E09F938F931F930E940F
:1027F000960888E28093E8030F900F900F900F9057
:102800000F908091180499279F938F9384E793E00A
:102810008BC01092E80383E893E09F938F931F93FC
:102820000E94960884E18093E8030F900F900F9028
:1028300080912304909124049F938F9382E993E0E5
:102840009F938F931F930E94960888E28093E803DA
:102850000F900F900F900F900F9080912704909100
:1028600028049F938F9381EA93E09F938F931F9304
:102870000E9496088CE38093E8030F900F900F90CE
:102880000F900F9080912504909126049F938F9331
:1028900080EB93E049C01092E80380911F0490916F
:1028A00020049F938F938FEB93E09F938F931F93BD
:1028B0000E94960884E18093E8030F900F900F9098
:1028C0000F900F9080911D0490911E049F938F9301
:1028D0008BEC93E09F938F931F930E94960888E25E
:1028E0008093E8030F900F900F900F900F908091BE
:1028F0001B0490911C049F938F9387ED93E09F930B
:102900008F931F930E9496088CE38093E8030F90A7
:102910000F900F900F900F908091190490911A04CE
:102920009F938F9383EE93E09F938F931F930E94C7
:1029300096080F900F900F900F900F9057C0109225
:10294000E8038FEE93E09F938F931F930E94960866
:1029500084E18093E8030F900F900F9080917003B3
:1029600099279F938F9387EF93E09F938F931F9364
:102970000E94960888E28093E8030F900F900F90D2
:102980000F900F908091BD039091BE039F938F9302
:1029900085E094E09F938F931F930E9496088CE3A9
:1029A0008093E8030F900F900F900F900F908091FD
:1029B0005B0799279F938F9380915A0799279F933D
:1029C0008F9383E194E09F938F931F930E949608C7
:1029D0008DB79EB707960FB6F8949EBF0FBE8DBFFA
:1029E00005C0815080936A031092EB031092E703B5
:1029F000DF91CF911F9108951092B9008AE28093E0
:102A0000B800089585EA8093BC0080E090E00895C6
:102A100084E98093BC0008951092B9008093BB00B4
:102A200085E88093BC0080E090E008950E9408153E
:102A30001092EE038091BB001092ED0380E880932A
:102A4000BC001092BD001092BA001092BB00109210
:102A5000B9001092B8000E94FC140E94021580E098
:102A60000E940C1508951F920F920FB60F92112419
:102A70002F933F934F935F936F937F938F939F9386
:102A8000AF93BF93EF93FF938091EE03282F3327EB
:102A90008F5F8093EE032330310509F446C0243064
:102AA00031054CF421303105D1F0223031057CF56F
:102AB000232B81F083C025303105E1F1253031052C
:102AC0000CF441C026303105F1F12730310509F40D
:102AD0005AC074C08091ED03880F8E5A51C0809106
:102AE000ED03282F33278F5F8093ED0321303105CD
:102AF00009F43EC0223031051CF4232BB1F15EC035
:102B000022303105C1F123303105C1F157C00E9497
:102B100008158091ED03843018F41092EE0302C082
:102B20001092ED030E94021549C08091EC03880FBA
:102B30008D5A26C08091EC03E82FFF27ED5FF84FF8
:102B40008091BB0080838091EC03992781309105AF
:102B500079F0823091051CF4892B39F02FC0823036
:102B6000910549F0039751F029C08091810708C071
:102B70008091860705C080919E0702C08091A007C2
:102B80000E940C151BC09091EC03E92FFF27ED5F0D
:102B9000F84F8091BB008483892F8F5F8093EC0373
:102BA000843010F01092EC030E9408158AE090E047
:102BB00090938703809386031092EE038091BC006C
:102BC00080688093BC00FF91EF91BF91AF919F917E
:102BD0008F917F916F915F914F913F912F910F90C6
:102BE0000FBE0F901F90189583EC80938100809109
:102BF0006F00806280936F001092740410927304CF
:102C00001092760410927504109278041092770452
:102C100008951F920F920FB60F9211242F933F9396
:102C20004F935F936F937F938F939F93AF93BF93D4
:102C3000EF93FF9340918600509187008091EF03BE
:102C40009091F003481B590B80918600909187006A
:102C50009093F0038093EF03CA018D549440209128
:102C6000F1033091F203835F9A4160F4243031051F
:102C700014F010926B0381E090E09093F203809344
:102C8000F1036BC02A3031050CF067C0CA018B5FBD
:102C90009040845B914008F043C0425D5140F9018F
:102CA000E20FF31FE55FF84F80819181BA01681B45
:102CB000790BCB0177FF03C0909581959F4F0697C5
:102CC0004CF480911804883C28F480911804865FA5
:102CD00080931804F901E20FF31FDF01A55FB84FDD
:102CE0008D919C9111979C01220F331F280F391F42
:102CF000240F351F37FF02C02D5F3F4FC901959547
:102D0000879595958795EF5DF84F2D913C9111979B
:102D1000AC01421B530B5183408311969C938E93BD
:102D20008091F1039091F20301969093F2038093C6
:102D3000F103059711F45D9A01C05D988091F1034C
:102D40009091F2038630910511F45C9A01C05C9871
:102D5000079711F45B9A01C05B98FF91EF91BF91C7
:102D6000AF919F918F917F916F915F914F913F9123
:102D70002F910F900FBE0F901F90189581E08093B8
:102D8000370782E08093380783E08093390734E087
:102D900030933A0765E060933B0786E080933C07F9
:102DA00087E080933D0798E090933E0780E480930E
:102DB0003F078EE1809340078BEF809342075AE0F4
:102DC0005093430722E32093410720934507309314
:102DD000440730934607909347078EE08093480757
:102DE0008FE0809349078AEF80934A078AE18093B6
:102DF0004B0790E890934C0788E780934D0746E98E
:102E000040934E078EE580934F0783E280935007EF
:102E100084E1809351071092520780E28093530718
:102E20009093540710925507109256071092570727
:102E300010926707109268071092690710926A074C
:102E400094E69093580788E28093590710926C0794
:102E500020935A0740935B0760935C0720935D07BC
:102E60008AE580935E0720935F0710926B0790932B
:102E700060075093610790936207909363072093D4
:102E800064073093650790936607A1E7B7E0E8E829
:102E9000F3E08CE001900D928150E1F7089581E01C
:102EA0008093370792E09093380783E08093390747
:102EB00044E040933A0755E050933B0786E0809307
:102EC0003C0787E080933D0788E080933E0780E4DD
:102ED00080933F078EE1809340078BEF80934207FA
:102EE0003AE03093430722E32093410720934507BC
:102EF0009093440740934607109247073093480742
:102F00008FE0809349078AEF80934A078AE1809394
:102F10004B0780E880934C078FEA80934D0780939E
:102F20004E078EE580934F0783E28093500784E13C
:102F3000809351071092520780E28093530780E5F7
:102F40008093540710925507109256071092570716
:102F500010926707109268071092690710926A072B
:102F600094E69093580788E28093590710926C0773
:102F700020935A0786E980935B0750935C07209360
:102F80005D078AE580935E0720935F0710926B07C9
:102F90009093600730936107909362079093630763
:102FA00090936407409365078BE480936607A1E7DD
:102FB000B7E0EFE8F3E08CE001900D928150E1F78B
:102FC000089581E08093370762E06093380753E00B
:102FD00050933907E4E0E0933A0775E070933B07BC
:102FE00086E080933C0787E080933D0738E030938C
:102FF0003E0781EC80933F078EE18093400724E6F3
:10300000209342074AE04093430792E3909341079D
:1030100090934507609344075093460710924707E3
:10302000309348078FE0809349078AEF80934A07DF
:103030008AE180934B0780E880934C0788EC80936B
:103040004D078FEA80934E078EE580934F0783E20A
:103050008093500784E18093510710925207409368
:10306000530780E580935407109255071092560736
:10307000109257071092670710926807109269071D
:1030800010926A072093580788E28093590710929C
:103090006C0790935A0786E980935B0770935C07EF
:1030A00090935D078AE580935E0790935F07109287
:1030B0006B0720936007409361072093620720937A
:1030C000630720936407E093650790936607A1E781
:1030D000B7E0E7E9F3E08CE001900D928150E1F771
:1030E0000895CF93C82FC150CF3F81F08091110434
:1030F000882361F484E690E09093C0038093BF033B
:103100008AEF90E00E94090CC15080F7CF9108959A
:1031100010927A008091DD039091DE0390938807EE
:10312000809387078091DB039091DC039093800765
:1031300080937F078091D9039091DA039093A7073A
:103140008093A6078091D5039091D603AA2797FD77
:10315000A095BA2FBC01CD012CE030E040E050E05A
:103160000E944E3CDC01CB019093A4078093A307FF
:103170008091D7039091D803AA2797FDA095BA2FE5
:10318000BC01CD010E944E3CDC01CB019093AE0707
:103190008093AD078091D3039091D40390938F07D0
:1031A00080938E078FEE80937A0080913B07E82F03
:1031B000FF27EE0FFF1FE55FF84F80819181825955
:1031C0009F4F20911F0430912004281739071CF4C9
:1031D0002F5F3F4F0CC08081918182599F4F821792
:1031E00093074CF42115310531F0215030403093D4
:1031F000200420931F0480913C07E82FFF27EE0F47
:10320000FF1FE55FF84F8081918182599F4F209188
:103210001D0430911E04281739071CF42F5F3F4FFF
:103220000CC08081918182599F4F821793074CF483
:103230002115310531F02150304030931E04209388
:103240001D0480913D07E82FFF27EE0FFF1FE55F6C
:10325000F84F8081918182599F4F20911B043091BA
:103260001C04281739071CF42F5F3F4F0CC08081C6
:10327000918182599F4F821793074CF42115310594
:1032800031F02150304030931C0420931B04809176
:103290003E07E82FFF27EE0FFF1FE55FF84F808105
:1032A000918182599F4F2091190430911A04281757
:1032B00039071CF42F5F3F4F0CC0808191818259E8
:1032C0009F4F821793074CF42115310531F021509F
:1032D000304030931A042093190480911F04909178
:1032E000200497FF05C01092200410921F040AC00A
:1032F0008F3F910539F034F08FEF90E090932004E8
:1033000080931F0480911D0490911E0497FF05C0B7
:1033100010921E0410921D040AC08F3F910539F0CF
:1033200034F08FEF90E090931E0480931D04809101
:103330001B0490911C0497FF05C010921C0410926E
:103340001B040AC08F3F910539F034F08FEF90E0F5
:1033500090931C0480931B048091190490911A048B
:1033600097FF05C010921A04109219040AC08F3FEB
:10337000910539F034F08FEF90E090931A04809328
:103380001904809162079927AA27BB27BC01CD01A8
:1033900024EC39E040E050E00E944E3CDC01CB01DF
:1033A0008093820390938303A0938403B093850357
:1033B00080937E0390937F03A0938003B093810357
:1033C000089510926E0410926D0410926C04109285
:1033D0006B0480E090E0A0E0B0E0809367049093FD
:1033E0006804A0936904B0936A0410927804109260
:1033F000770410927604109275041092740410925F
:1034000073041092FA031092F9030E94881884E65C
:1034100090E00E94160C0E94881880913F0780FF60
:1034200010C08091080390910903875B934038F4A2
:1034300080910803909109038E5E924010F40E94DF
:10344000E40C8091DD039091DE03909378048093E7
:1034500077048091DB039091DC0390937604809352
:1034600075048091D9039091DA039093740480934A
:103470007304809175049091760490937204809304
:1034800071048091770490917804909370048093F4
:103490006F0444E050E0DA010E94DD3C802D85306D
:1034A00078F18091AD079091AE078091AD07909132
:1034B000AE0797FF03C0909581959F4F6CE070E039
:1034C0000E948D3C70936C0460936B048091A30701
:1034D0009091A4078091A3079091A40797FF03C040
:1034E000909581959F4F6CE070E00E948D3C7093A9
:1034F0006E0460936D048091F3069091F40634C0DD
:10350000DA010E94DD3C802D9927982F8827DA0167
:1035100011960E94DD3C202D820F911D90936E0428
:1035200080936D04DA0112960E94DD3C802D99276C
:10353000982F8827DA0113960E94DD3C202D820FF8
:10354000911D90936C0480936B04DA0114960E9491
:10355000DD3C802D9927982F8827DA0115960E9447
:10356000DD3C202D820F911DAA2797FDA095BA2F33
:10357000BC01CD010E948C3BDC01CB018093670430
:1035800090936804A0936904B0936A041092410474
:1035900010924204109243041092440410923D048D
:1035A00010923E0410923F0410924004109239048D
:1035B00010923A0410923B0410923C04109235048D
:1035C000109236041092370410923804109231048D
:1035D000109232041092330410923404109288072F
:1035E000109287071092800710927F071092A7070A
:1035F0001092A60780910A0390910B03A0910C03EF
:10360000B0910D039093F6068093F5061092CC03CB
:103610001092CB031092290410922A0410922B04CA
:1036200010922C04809127049091280490932604F2
:10363000809325040E94AF3A82E390E09093C00308
:103640008093BF03809162079927AA27BB27BC01FB
:10365000CD0124EC39E040E050E00E944E3CDC011A
:10366000CB018093820390938303A0938403B09350
:103670008503809163079927AA27BB27BC01CD0149
:103680000E944E3CDC01CB0180937E0390937F032C
:10369000A0938003B093810310926D0310926C038A
:1036A0000895AF92BF92CF92DF92EF92FF920F9365
:1036B0001F93CF93DF9380917304909174042091B2
:1036C000D9033091DA03821B930B9093A707809361
:1036D000A6078091DB039091DC0320917504309163
:1036E0007604821B930B9093800780937F078091D1
:1036F000DD039091DE032091770430917804821BE2
:10370000930B90938807809387078091A3079091EC
:10371000A4077C010027F7FC0095102F8091D503AA
:103720009091D603AA2797FDA095BA2FBC01CD0191
:103730002CE030E040E050E00E944E3CDC01CB0148
:10374000E80EF91E0A1F1B1F17FF05C00894E11C95
:10375000F11C011D111D15950795F794E794F09242
:10376000A407E092A3078091AD079091AE077C017A
:103770000027F7FC0095102F8091D7039091D80374
:10378000AA2797FDA095BA2FBC01CD012CE030E00F
:1037900040E050E00E944E3CDC01CB01E80EF91EF7
:1037A0000A1F1B1F17FF05C00894E11CF11C011D17
:1037B000111D15950795F794E794F092AE07E092E6
:1037C000AD0780918E0790918F079C01442737FDAC
:1037D0004095542F8091D3039091D403AA2797FD4D
:1037E000A095BA2F280F391F4A1F5B1F57FF04C02F
:1037F0002F5F3F4F4F4F5F4F559547953795279513
:1038000030938F0720938E078091D5039091D60334
:103810006CE070E0869F9001879F300D969F300D81
:103820001124C9019C01442737FD4095542F8091F4
:10383000510490915204A0915304B0915404820F0A
:10384000931FA41FB51F8093510490935204A0931B
:103850005304B09354048091D7039091D803869F6A
:103860009001879F300D969F300D1124C9019C0156
:10387000442737FD4095542F80914D0490914E047C
:10388000A0914F04B0915004820F931FA41FB51F45
:1038900080934D0490934E04A0934F04B093500432
:1038A0008091490490914A04A0914B04B0914C043A
:1038B000BC01CD010E948C3B5B016C018091F30641
:1038C0009091F406AA2797FDA095BA2FBC01CD01CF
:1038D0000E948C3B7B018C0180916704909168046D
:1038E000A0916904B0916A049C01AD01C801B701BF
:1038F0000E94E63ADC01CB019C01AD01C601B50195
:103900000E94E73ADC01CB01BC01CD010E946F3B74
:10391000DC01CB018093490490934A04A0934B04AB
:10392000B0934C048091A6079091A7079C0144276F
:1039300037FD4095542F8091310490913204A0912D
:103940003304B0913404820F931FA41FB51F8093DA
:10395000310490933204A0933304B09334048091E3
:10396000A6079091A7079C01442737FD4095542F47
:1039700080912D0490912E04A0912F04B0913004D9
:10398000820F931FA41FB51F80932D0490932E04C4
:10399000A0932F04B0933004A0900804AA2009F04B
:1039A000A2C080910704882309F09DC080913F0741
:1039B00086FF99C0A0914104B0914204C091430494
:1039C000D0914404D7FF04C0A150B04FCF4FDF4F78
:1039D0003CE0D595C795B795A7953A95D1F78091D5
:1039E000A6079091A7079C01442737FD4095542FC7
:1039F000BD01CE010E944E3CDC01CB012091FA03B7
:103A0000E22EFF2400271127BC01CD01A801970158
:103A10000E944E3CDC01CB018093790490937A04A0
:103A2000A0937B04B0937C04B7FF04C08150984FEF
:103A3000AF4FBF4F2BE0B595A795979587952A95E2
:103A4000D1F78093790490937A04A0937B04B09388
:103A50007C04A0913904B0913A04C0913B04D09108
:103A60003C04D7FF04C0A150B04FCF4FDF4F8CE0D4
:103A7000D595C795B795A7958A95D1F78091A60753
:103A80009091A7079C01442737FD4095542FBD0115
:103A9000CE010E944E3CDC01CB01BC01CD01A8014E
:103AA00097010E944E3CDC01CB0180937D049093F2
:103AB0007E04A0937F04B0938004B7FF04C08150BC
:103AC000984FAF4FBF4F1BE0B595A795979587953A
:103AD0001A95D1F780937D0490937E04A0937F0480
:103AE000B093800410C010927D0410927E04109256
:103AF0007F04109280041092790410927A0410923C
:103B00007B0410927C0480917F0790918007209124
:103B1000790430917A04820F931F909380078093E9
:103B20007F070091F903202F3327442755278091E1
:103B30007D0490917E04A0917F04B0918004BC012B
:103B4000CD010E944E3C9B01AC0197FF04C0215067
:103B50003E4F4F4F5F4FC9E0559547953795279595
:103B6000CA95D1F780917F0790918007820F931FAC
:103B70009093800780937F0780917F0790918007C3
:103B80009C01442737FD4095542F80913504909136
:103B90003604A0913704B0913804820F931FA41FFC
:103BA000B51F8093350490933604A0933704B093E7
:103BB000380480917F079091800720910B04309109
:103BC0000C04821B930B9C01442737FD4095542F16
:103BD0008091390490913A04A0913B04B0913C0447
:103BE000820F931FA41FB51F8093390490933A044A
:103BF000A0933B04B0933C048091390490913A0423
:103C0000A0913B04B0913C04C0917E03D0917F030E
:103C1000E0918003F0918103C817D907EA07FB07F9
:103C200004F580E197E2A0E0B0E08C1B9D0BAE0BA9
:103C3000BF0B8093390490933A04A0933B04B09354
:103C40003C048091390490913A04A0913B04B091D6
:103C50003C048093350490933604A0933704B093CA
:103C6000380422273327A9012C1B3D0B4E0B5F0B79
:103C70008091390490913A04A0913B04B0913C04A6
:103C800082179307A407B507E4F4C051D742E04078
:103C9000F040C0933904D0933A04E0933B04F0938E
:103CA0003C048091390490913A04A0913B04B09176
:103CB0003C048093350490933604A0933704B0936A
:103CC00038048091DB039091DC030F9734F488E192
:103CD0009CEF9093800780937F078091DB03909106
:103CE000DC03079734F480E398EF90938007809388
:103CF0007F07109100011A30A9F48091DB039091A5
:103D0000DC03835F934034F088EE93E09093800768
:103D100080937F078091DB039091DC038A5F93405F
:103D2000DCF014C08091DB039091DC03855E97404A
:103D300034F088EE93E09093800780937F07809122
:103D4000DB039091DC03835F974034F080ED97E0D4
:103D50009093800780937F078091870790918807D1
:103D600020917D0430917E04821B930B90938807F1
:103D700080938707202F3327442755278091790484
:103D800090917A04A0917B04B0917C04BC01CD0198
:103D90000E944E3C9B01AC0197FF04C021503E4F56
:103DA0004F4F5F4FB9E05595479537952795BA9591
:103DB000D1F78091870790918807821B930B90938E
:103DC00088078093870780918707909188079C01D7
:103DD000442737FD4095542F80913D0490913E0437
:103DE000A0913F04B0914004820F931FA41FB51F00
:103DF00080933D0490933E04A0933F04B09340040D
:103E000080918707909188072091090430910A04D6
:103E1000821B930B9C01442737FD4095542F8091C2
:103E2000410490914204A0914304B0914404820F54
:103E3000931FA41FB51F8093410490934204A09345
:103E40004304B09344048091410490914204A091B2
:103E50004304B0914404C0918203D0918303E09164
:103E60008403F0918503C817D907EA07FB0704F517
:103E700080E197E2A0E0B0E08C1B9D0BAE0BBF0B86
:103E80008093410490934204A0934304B09344046C
:103E90008091410490914204A0914304B091440464
:103EA00080933D0490933E04A0933F04B09340045C
:103EB00022273327A9012C1B3D0B4E0B5F0B809152
:103EC000410490914204A0914304B09144048217AC
:103ED0009307A407B507E4F4C051D742E040F0408F
:103EE000C0934104D0934204E0934304F09344040C
:103EF0008091410490914204A0914304B091440404
:103F000080933D0490933E04A0933F04B0934004FB
:103F10008091DD039091DE030F9734F488E19CEFEC
:103F200090938807809387078091DD039091DE034B
:103F3000079734F480E398EF90938807809387077E
:103F40001A30A9F48091DD039091DE03835F9340E2
:103F500034F088EE93E090938807809387078091F0
:103F6000DD039091DE038A5F9340DCF014C0809102
:103F7000DD039091DE03855E974034F088EE93E098
:103F800090938807809387078091DD039091DE03EB
:103F9000835F974034F080ED97E09093880780939B
:103FA00087078FEE80937A008091310490913204DC
:103FB000A0913304B0913404809345049093460457
:103FC000A0934704B0934804809141049091420427
:103FD000A0914304B09144048093610490936204DF
:103FE000A0936304B09364048091390490913A04DF
:103FF000A0913B04B0913C048093590490935A04DF
:10400000A0935B04B0935C0480913D0490913E04C6
:10401000A0913F04B091400480935D0490935E04AE
:10402000A0935F04B09360048091350490913604AE
:10403000A0913704B09138048093550490935604AE
:10404000A0935704B093580480913F0787FF6EC038
:10405000AA2009F06BC080910704882309F066C08C
:104060008091870790918807893C91058CF0209179
:10407000870730918807220F331F220F331F80914B
:10408000870790918807820F931F8052934017C033
:10409000809187079091880788539F4FA4F42091BF
:1040A000870730918807220F331F220F331F80911B
:1040B000870790918807820F931F805E9C4F909393
:1040C00088078093870780917F0790918007893CBC
:1040D00091058CF020917F0730918007220F331FCC
:1040E000220F331F80917F0790918007820F931FCB
:1040F0008052934017C080917F079091800788532A
:104100009F4FA4F420917F0730918007220F331F27
:10411000220F331F80917F0790918007820F931F9A
:10412000805E9C4F9093800780937F0780913B0730
:10413000E82FFF27EE0FFF1FE55FF84F8081918189
:1041400082599F4F20911F0430912004281739076E
:104150001CF42F5F3F4F0CC08081918182599F4F8B
:10416000821793074CF42115310531F0215030406E
:104170003093200420931F0480913C07E82FFF27F1
:10418000EE0FFF1FE55FF84F8081918182599F4FAD
:1041900020911D0430911E04281739071CF42F5F4D
:1041A0003F4F0CC08081918182599F4F82179307A6
:1041B0004CF42115310531F02150304030931E046C
:1041C00020931D0480913D07E82FFF27EE0FFF1F6E
:1041D000E55FF84F8081918182599F4F20911B04A8
:1041E00030911C04281739071CF42F5F3F4F0CC077
:1041F0008081918182599F4F821793074CF421153A
:10420000310531F02150304030931C0420931B04C1
:1042100080913E07E82FFF27EE0FFF1FE55FF84F65
:104220008081918182599F4F2091190430911A0405
:10423000281739071CF42F5F3F4F0CC080819181F4
:1042400082599F4F821793074CF42115310531F0A5
:104250002150304030931A042093190480911F0498
:104260009091200497FF05C01092200410921F0423
:104270000AC08F3F910539F034F08FEF90E09093B2
:10428000200480931F0480911D0490911E0497FFC9
:1042900005C010921E0410921D040AC08F3F9105A4
:1042A00039F034F08FEF90E090931E0480931D045A
:1042B00080911B0490911C0497FF05C010921C0470
:1042C00010921B040AC08F3F910539F034F08FEF34
:1042D00090E090931C0480931B04809119049091AA
:1042E0001A0497FF05C010921A04109219040AC00C
:1042F0008F3F910539F034F08FEF90E090931A04DE
:1043000080931904DF91CF911F910F91FF90EF904F
:10431000DF90CF90BF90AF900895809111048823D3
:1043200001F5809386078093810780939E07809391
:10433000A0078091A503882311F0809381078091C5
:10434000A603882311F0809386078091A703882312
:1043500011F08093A0078091A803882311F0809327
:104360009E078091810799279093C9068093C8067C
:104370008091860799279093CB068093CA068091F7
:10438000A00799279093CD068093CC0680919E0735
:1043900099279093CF068093CE061092EE03109249
:1043A000ED030E94021508951F93809142078B3FF1
:1043B00098F08B3F19F480911F040EC08C3F19F4C4
:1043C00080911D0409C08D3F19F480911B0404C025
:1043D0008E3F21F4809119048093780380917803B3
:1043E000882321F08F3F11F4809378038091410757
:1043F0008B3F98F08B3F19F480911F040EC08C3FC7
:1044000019F480911D0409C08D3F19F480911B049B
:1044100004C08E3F21F48091190480937903809128
:104420007903882329F0843618F084E68093790391
:10443000809143078B3F98F08B3F19F480911F04C4
:104440000EC08C3F19F480911D0409C08D3F19F4F2
:1044500080911B0404C08E3F21F480911904809345
:10446000770380917703882329F0843618F084E657
:1044700080937703809145078B3F98F08B3F19F429
:1044800080911F040EC08C3F19F480911D0409C057
:104490008D3F19F480911B0404C08E3F21F480915C
:1044A00019048093760380917603882321F08F3F4F
:1044B00011F48093760380914C078B3F98F08B3FEB
:1044C00019F480911F040EC08C3F19F480911D04D3
:1044D00009C08D3F19F480911B0404C08E3F21F464
:1044E000809119048093750380917503882321F0CE
:1044F0008F3F11F48093750380914D078B3F98F0A7
:104500008B3F19F480911F040EC08C3F19F48091E9
:104510001D0409C08D3F19F480911B0404C08E3F17
:1045200021F48091190480937403809174038B307B
:1045300010F48AE002C08F3F11F4809374038091DD
:104540004E078B3F98F08B3F19F480911F040EC0EB
:104550008C3F19F480911D0409C08D3F19F480919E
:104560001B0404C08E3F21F48091190480937303CF
:1045700080917303882321F08F3F11F4809373039C
:10458000809153078B3F98F08B3F19F480911F0463
:104590000EC08C3F19F480911D0409C08D3F19F4A1
:1045A00080911B0404C08E3F21F4809119048093F4
:1045B000710380917103882321F08F3F11F4809360
:1045C0007103809154078B3F98F08B3F19F48091D1
:1045D0001F040EC08C3F19F480911D0409C08D3F4B
:1045E00019F480911B0404C08E3F21F480911904BA
:1045F0008093020480910204882321F08F3F11F4FC
:1046000080930204809155078B3F98F08B3F19F4FB
:1046100080911F040EC08C3F19F480911D0409C0C5
:104620008D3F19F480911B0404C08E3F21F48091CA
:1046300019048093010480910104882321F08F3FA5
:1046400011F480930104809156078B3F98F08B3FC3
:1046500019F480911F040EC08C3F19F480911D0441
:1046600009C08D3F19F480911B0404C08E3F21F4D2
:10467000809119048093000480910004882321F024
:104680008F3F11F480930004809157078B3F98F07F
:104690008B3F19F480911F040EC08C3F19F4809158
:1046A0001D0409C08D3F19F480911B0404C08E3F86
:1046B00021F4809119048093FF038091FF038823E4
:1046C00021F08F3F11F48093FF03809167078B3FA8
:1046D00098F08B3F19F480911F040EC08C3F19F4A1
:1046E00080911D0409C08D3F19F480911B0404C002
:1046F0008E3F21F4809119048093FE038091FE0384
:10470000882321F08F3F11F48093FE038091680786
:104710008B3F98F08B3F19F480911F040EC08C3FA3
:1047200019F480911D0409C08D3F19F480911B0478
:1047300004C08E3F21F4809119048093FD03809181
:10474000FD03882321F08F3F11F48093FD038091B6
:1047500069078B3F98F08B3F19F480911F040EC0BE
:104760008C3F19F480911D0409C08D3F19F480918C
:104770001B0404C08E3F21F4809119048093FC0334
:104780008091FC03882321F08F3F11F48093FC0378
:1047900080916A078B3F98F08B3F19F480911F043A
:1047A0000EC08C3F19F480911D0409C08D3F19F48F
:1047B00080911B0404C08E3F21F4809119048093E2
:1047C000FB038091FB03882321F08F3F11F480933A
:1047D000FB03809158078B3F98F08B3F19F4809131
:1047E0001F040EC08C3F19F480911D0409C08D3F39
:1047F00019F480911B0404C08E3F21F480911904A8
:104800008093700380917003882321F08F3F11F40F
:104810008093700380915D078B3F98F08B3F19F474
:1048200080911F040EC08C3F19F480911D0409C0B3
:104830008D3F19F480911B0404C08E3F21F48091B8
:10484000190480936F0380916F03882321F08F3FB9
:1048500011F480936F03809160078B3F98F08B3F3A
:1048600019F480911F040EC08C3F19F480911D042F
:1048700009C08D3F19F480911B0404C08E3F21F4C0
:10488000809119048093FA038091FA03882321F020
:104890008F3F11F48093FA03809161078B3F98F06A
:1048A0008B3F19F480911F040EC08C3F19F4809146
:1048B0001D0409C08D3F19F480911B0404C08E3F74
:1048C00021F4809119048093F9038091F9038823DE
:1048D00021F08F3F11F48093F903809166078B3F9D
:1048E00098F08B3F19F480911F040EC08C3F19F48F
:1048F00080911D0409C08D3F19F480911B0404C0F0
:104900008E3F21F48091190480936E0380916E0391
:10491000882321F08F3F11F480936E03109171036F
:10492000812F992787FD9095A92FB92FBC01CD0123
:104930000E948C3B17FF06C020E030E040E853E4C3
:104940000E94E73A27E137EB41ED58E30E94063C2D
:10495000DC01CB0180937A0390937B03A0937C03CB
:10496000B0937D0380914A078093A5078091490702
:10497000809389071F9108952F923F924F925F92E3
:104980006F927F928F929F92AF92BF92CF92DF925F
:10499000EF92FF920F931F93CF93DF93CDB7DEB7C4
:1049A0002B970FB6F894DEBF0FBECDBF0E94511BF0
:1049B000299A80913907E82FFF27EE0FFF1FE55F47
:1049C000F84F6080718028E730E0620E731E80919E
:1049D000A50799274497861597050CF43C0177FEA7
:1049E00002C06624772480911804843608F05EC0E3
:1049F00080910103882399F4809104039091050329
:104A00008F5F9F4F61F488E99AE39093C00380938E
:104A1000BF0380E09CE090930503809304038091A2
:104A20009D0490919E04009731F0019790939E040D
:104A300080939D0404C0109211041092220480916E
:104A400000018A3011F4289A01C028988091A204AC
:104A50009091A304815D974030F180915007682EBA
:104A6000772481E08093220480913707E82FFF2785
:104A7000EE0FFF1FE55FF84F11821082809138071B
:104A8000E82FFF27EE0FFF1FE55FF84F118210821E
:104A900080913A07E82FFF27EE0FFF1FE55FF84FE1
:104AA000118210825BC21092110458C280911804C6
:104AB0008D3808F453C2109222049091510782E37A
:104AC000989FC001112490939E0480939D0459E205
:104AD000651671046CF08091A2049091A3046FEFAD
:104AE0008F3F960729F001969093A3048093A20428
:104AF0008091A2049091A304883C910520F078E273
:104B00006716710404F510928104109282041092C9
:104B100083041092840410928504109286041092EB
:104B2000870410928804109231041092320410927B
:104B300033041092340410922D0410922E0410921B
:104B40002F041092300489EC681671040CF466C1CD
:104B500020911104222309F061C180913A07E82FC6
:104B6000FF27EE0FFF1FE55FF84F808191818C34A6
:104B700091050CF4CAC080919F048F5F80939F04BD
:104B8000893C08F44BC1299820939F041092A304F8
:104B90001092A20430913707E32FFF27EE0FFF1F7B
:104BA000E55FF84F8081918187349105B4F480915D
:104BB0003807E82FFF27EE0FFF1FE55FF84F8081D2
:104BC00091810190F081E02DF7FF03C0F095E19510
:104BD000FF4FE734F1050CF47AC041E0209138072B
:104BE000A22FBB27AA0FBB1FA55FB84F8D919C9129
:104BF00011978734910544F0E32FFF27EE0FFF1F35
:104C0000E55FF84F808191818D919C91873491056A
:104C100074F080913707E82FFF27EE0FFF1FE55F45
:104C2000F84F80819181873491050CF042E0E22FAA
:104C3000FF27EE0FFF1FE55FF84F808191818634DB
:104C4000910574F480913707E82FFF27EE0FFF1FBF
:104C5000E55FF84F80819181873491050CF043E046
:104C6000E22FFF27EE0FFF1FE55FF84F8081918154
:104C70008A5B9F4F74F480913707E82FFF27EE0F70
:104C8000FF1FE55FF84F80819181873491050CF01B
:104C900044E0E22FFF27EE0FFF1FE55FF84F808112
:104CA00091818A5B9F4F74F480913707E82FFF272B
:104CB000EE0FFF1FE55FF84F8081918186349105EB
:104CC0000CF445E0A2E0B0E0042E0E94E53C8091A7
:104CD0003F0780FF10C08091080390910903875B14
:104CE000934038F480910803909109038E5E9240BE
:104CF00010F40E94E40C0E94580247E467E377E056
:104D00000E942E020E94E11982C080819181855B00
:104D10009F4F0CF081C080919F048F5F80939F0410
:104D2000893C08F47BC02998A4E0B0E08FEF082EFE
:104D30000E94E53C2093110420939F041092A30449
:104D40001092A2040E94E119A4E0B0E080916D04E9
:104D500090916E0497FF02C081509F4F892F990F49
:104D6000990B082E0E94E53CA5E0B0E080916D040F
:104D700090916E04082E0E94E53CA6E0B0E0809180
:104D80006B0490916C0497FF02C081509F4F892F54
:104D9000990F990B082E0E94E53CA7E0B0E08091A6
:104DA0006B0490916C04082E0E94E53C08E010E032
:104DB0008091670490916804A0916904B0916A049D
:104DC000BC01CD010E946F3BDC01CB019C0197FF30
:104DD00002C021503F4F832F992787FD9A95D80114
:104DE000082E0E94E53C09E010E080916704909154
:104DF0006804A0916904B0916A04BC01CD010E94CD
:104E00006F3BDC01CB01D801082E0E94E53C0E94DB
:104E100058020E94711802C020939F04B3E26B16DF
:104E200071040CF09BC020913A07E22FFF27EE0F90
:104E3000FF1FE55FF84F80819181855B9F4F0CF0EC
:104E40006DC08091A0048F5F8093A004893C08F41A
:104E500067C088EC8093A00481E090E09093A30465
:104E60008093A20481E0809311041092890410922F
:104E70008A0410928B0410928C04109231041092C8
:104E80003204109233041092340410922D041092C4
:104E90002E0410922F0410923004109241041092AC
:104EA0004204109243041092440410923904109268
:104EB0003A0410923B0410923C048091610490915A
:104EC0006204A0916304B091640480933D049093C4
:104ED0003E04A0933F04B093400480915904909104
:104EE0005A04A0915B04B0915C04809335049093C4
:104EF0003604A0933704B0933804109281041092C2
:104F000082041092830410928404109285041092FB
:104F10008604109287041092880402C01092A004A4
:104F2000E22FFF27EE0FFF1FE55FF84F8081918191
:104F30008C3491058CF08091A1048F5F8093A10443
:104F4000893C60F01092110488EC8093A1041092C7
:104F5000A3041092A20402C01092A10480916B03DA
:104F6000815080936B0380916B038F3F29F0809178
:104F70002204882309F492C30E94D421E0903707C9
:104F8000EE2DFF27EE0FFF1FDF01A55FB84F009149
:104F90004607602F77278D919C91869F9001879F70
:104FA000300D969F300D1124EF5DF84F809147072B
:104FB000482F552780819181849FD001859FB00D16
:104FC000949FB00D11242A0F3B1F30931704209398
:104FD0001604F0903807EF2DFF27EE0FFF1FDF01BB
:104FE000A55FB84F8D919C91869F9001879F300D52
:104FF000969F300D1124EF5DF84F80819181849F41
:10500000F001859FF00D949FF00D11242E0F3F1F8E
:10501000309315042093140480913A07E82FFF275A
:10502000EE0FFF1FE55FF84F80819181909581958C
:105030009F4F909313048093120410917403812F57
:10504000992787FD9095A92FB92FBC01CD010E940A
:105050008C3B17FF06C020E030E040E853E40E949C
:10506000E73A20E030E040E251E40E94E73ADC0118
:10507000CB0120E030E040E85BE3BC01CD010E94C1
:10508000063CDC01CB018093A8079093A907A0936D
:10509000AA07B093AB0710917303812F992787FD5F
:1050A0009095A92FB92FBC01CD010E948C3B17FF11
:1050B00006C020E030E040E853E40E94E73A20E0F8
:1050C00030EE4BE257E40E94293BDC01CB01809398
:1050D0009A0790939B07A0939C07B0939D076091BC
:1050E000A303662331F08AE090E09093C00380939D
:1050F000BF03462F552742FF09C080910204282F85
:105100003327220F331F220F331F13C09A01287039
:10511000307043FF0EC080910204282F33278CEF9C
:105120009FEF289FA001299F500D389F500D1124FB
:105130009A018091F7039091F803AC01A3E0440F2A
:10514000551FAA95E1F7481B590B420F531F57FFF4
:1051500002C0495F5F4FF3E055954795FA95E1F737
:105160005093F8034093F703462F552744FF09C097
:1051700080910204282F3327220F331F220F331F61
:1051800013C09A012072307045FF0EC08091020456
:10519000282F33278CEF9FEF289FB001299F700D98
:1051A000389F700D11249B018091F5039091F603B7
:1051B000AC0173E0440F551F7A95E1F7481B590B7A
:1051C000420F531F57FF02C0495F5F4F63E0559581
:1051D00047956A95E1F75093F6034093F5034091A4
:1051E000A203842F992783FF03C082E390E007C0C6
:1051F0009C012470307082FF07C08EEC9FEF90936B
:10520000F4038093F30304C03093F4032093F30377
:10521000242F332721FF09C080916C0390916D03E7
:10522000019690936D0380936C0324FF09C08091D5
:105230006C0390916D03019790936D0380936C03C1
:105240008091F7039091F80397FD079653E09595A9
:1052500087955A95E1F7C0901604D0901704C80EB0
:10526000D91ED0921704C09216042091F5033091F4
:10527000F60337FF02C0295F3F4F43E0359527957E
:105280004A95E1F78091140490911504820F931FC1
:105290009093150480931404809112049091130448
:1052A0002091F3033091F403820F931F9093130422
:1052B0008093120480913F0782FF0CC080E090E051
:1052C000A0E0B0E080939A0790939B07A0939C077F
:1052D000B0939D078091A8079091A907A091AA0774
:1052E000B091AB0720E030E040E050E0BC01CD01E0
:1052F0000E94963B882364F480E090E0A0E0B0E058
:105300008093A8079093A907A093AA07B093AB072F
:1053100080919A0790919B07A0919C07B0919D075F
:1053200020E030E040E050E0BC01CD010E94963B1F
:10533000882364F480E090E0A0E0B0E080939A07D6
:1053400090939B07A0939C07B0939D0710916B07C8
:10535000812F992782FDC8C083FDC6C0809161045A
:1053600090916204A0916304B091640481569A4EB6
:10537000A040B040ECF0602F7727CB0123E0880FEE
:10538000991F2A95E1F79601281B390B30931704D2
:10539000209316048091610490916204A0916304AB
:1053A000B091640481589843A140B040A4F128C052
:1053B0008091610490916204A0916304B0916404AF
:1053C000805A9541AF4FBF4F34F5602F77279B012F
:1053D00003E0220F331F0A95E1F72C0D3D1D30939A
:1053E0001704209316048091610490916204A091A7
:1053F0006304B091640481589843A140B0405CF0CC
:10540000B4E0660F771FBA95E1F7261B370B309390
:105410001704209316048091590490915A04A09186
:105420005B04B0915C0481569A4EA040B0401CF1E0
:1054300080914607482F5527CA01A3E0880F991F7E
:10544000AA95E1F72091140430911504281B390B1B
:1054500030931504209314048091590490915A04B8
:10546000A0915B04B0915C0481589843A140B04086
:105470000CF43AC02EC08091590490915A04A09126
:105480005B04B0915C04805A9541AF4FBF4F64F507
:1054900080914607482F5527CA01F3E0880F991FCE
:1054A000FA95E1F72091140430911504280F391F63
:1054B00030931504209314048091590490915A0458
:1054C000A0915B04B0915C0481589843A140B04026
:1054D0005CF0E4E0440F551FEA95E1F7241B350B1F
:1054E0003093150420931404EF2DFF27EE0FFF1FB8
:1054F000E55FF84F40915E07242F3327808191812B
:105500002817390734F412FF04C081E080930604A1
:1055100013C0EF2DFF27EE0FFF1FE55FF84F842F1D
:10552000992720915F07821B9109208131812817DB
:10553000390714F41092060440913807E42FFF272E
:10554000EE0FFF1FE55FF84F50915E07852F9927FB
:1055500022273327281B390B8081918182179307DB
:1055600044F480916B0783FF04C081E080930504BD
:1055700016C080910504882391F0E42FFF27EE0FD9
:10558000FF1FE55FF84F80915F079927851B910901
:10559000208131818217930714F410920504EE2DB7
:1055A000FF27EE0FFF1FE55FF84F40915E07242FA6
:1055B0003327808191812817390744F480916B0744
:1055C00080FF04C081E08093030417C0809103042E
:1055D000882399F0EE2DFF27EE0FFF1FE55FF84FB0
:1055E000842F992720915F07821B910920813181A7
:1055F0002817390714F41092030440913707E42F59
:10560000FF27EE0FFF1FE55FF84F50915E07852FD4
:10561000992722273327281B390B808191818217F4
:10562000930744F480916B0781FF04C081E080936D
:10563000040416C080910404882391F0E42FFF270E
:10564000EE0FFF1FE55FF84F80915F079927851BDD
:105650009109208131818217930714F41092040478
:1056600080910604882319F480910504811181E05A
:105670008093070480910304882321F4809104041B
:10568000882351F081E0809308041092070410925F
:1056900006041092050402C08093080420910704B8
:1056A000222331F084E690E09093C0038093BF03FF
:1056B000222321F480910804882339F080915D072A
:1056C0009927861597050CF43C01909022049920A7
:1056D00041F11092130410921204109217041092C8
:1056E000160410921504109214048DEC9CECACEC92
:1056F000BDE38093A8079093A907A093AA07B0934E
:10570000AB078AE097EDA3EABBE380939A079093F7
:105710009B07A0939C07B0939D07109207041092DB
:1057200008048091920790919307A0919407B091FB
:105730009507209161043091620440916304509177
:105740006404820F931FA41FB51F80939207909348
:105750009307A0939407B093950780919607909133
:105760009707A0919807B09199072091590430911B
:105770005A0440915B0450915C04820F931FA41F54
:10578000B51F8093960790939707A0939807B093BF
:10579000990780918A0790918B07A0918C07B0910F
:1057A0008D0720915D0430915E0440915F0450911B
:1057B0006004820F931FA41FB51F80938A079093E4
:1057C0008B07A0938C07B0938D07809182079091EF
:1057D0008307A0918407B0918507209155043091EB
:1057E00056044091570450915804820F931FA41FF0
:1057F000B51F8093820790938307A0938407B0938B
:10580000850780900804882029F480910704882364
:1058100009F45FC010925104109252041092530484
:105820001092540410924D0410924E0410924F04A2
:1058300010925004109292071092930710929407BE
:10584000109295071092960710929707109298075A
:105850001092990710928A0710928B0710928C076A
:1058600010928D071092820710928307109284077E
:10587000109285078091410490914204A0914304C5
:10588000B091440480933D0490933E04A0933F0460
:10589000B09340048091390490913A04A0913B0464
:1058A000B0913C048093350490933604A093370460
:1058B000B09338041092CA031092C90310920A04DC
:1058C0001092090410920C0410920B04882009F025
:1058D000BAC080910704882309F0B5C080914B07B6
:1058E000A82EBB24CC24DD24809161049091620415
:1058F000A0916304B0916404BC01CD01A60195019F
:105900000E94C23C79018A018091A3079091A4076B
:10591000AA2797FDA095BA2FE81AF90A0A0B1B0BC4
:10592000D801C70117FF03C00F96A11DB11D7C014F
:105930008D0174E015950795F794E7947A95D1F762
:105940008091590490915A04A0915B04B0915C0439
:10595000BC01CD01A60195010E94C23C8091AD071A
:105960009091AE07AA2797FDA095BA2F281B390B57
:105970004A0B5B0BDA01C90157FF03C00F96A11D4B
:10598000B11D9C01AD0164E055954795379527956C
:105990006A95D1F7F1E2EF16F104010511052CF03B
:1059A00090E2E92EF12C012D112D60EEE6166FEF3D
:1059B000F6066FEF06076FEF160744F480EEE82E49
:1059C0008FEFF82E8FEF082F8FEF182F2132310530
:1059D0004105510524F020E230E040E050E0203E57
:1059E0007FEF37077FEF47077FEF570724F420EE5D
:1059F0003FEF4FEF5FEF8091410490914204A091FF
:105A00004304B09144048E199F09A00BB10B8093FD
:105A1000410490934204A0934304B09344048091C2
:105A2000390490913A04A0913B04B0913C04821B4C
:105A3000930BA40BB50B8093390490933A04A09375
:105A40003B04B0933C048091C9039091CA038F3FFB
:105A5000910509F008F4C3C5882009F042C580917A
:105A60000704882309F03DC5809192079091930720
:105A7000A0919407B0919507B7FF04C081509F4F44
:105A8000AF4FBF4F892F9A2FAB2FBB27A7FDBA95DA
:105A90008093920790939307A0939407B0939507F0
:105AA0008091960790919707A0919807B0919907D8
:105AB000B7FF04C081509F4FAF4FBF4F892F9A2F20
:105AC000AB2FBB27A7FDBA958093960790939707B6
:105AD000A0939807B093990780914B07E82EFF2475
:105AE0000027112720915104309152044091530412
:105AF00050915404C801B7010E944E3C97FF04C066
:105B000061507F4F8F4F9F4FBB2797FDBA95A92FAD
:105B1000982F872F8093510490935204A09353049D
:105B2000B093540420914D0430914E0440914F04A1
:105B300050915004C801B7010E944E3C97FF04C029
:105B400061507F4F8F4F9F4FBB2797FDBA95A92F6D
:105B5000982F872F80934D0490934E04A0934F0469
:105B6000B09350048091490490914A04A0914B0451
:105B7000B0914C04B7FF04C081509F4FAF4FBF4F4F
:105B8000892F9A2FAB2FBB27A7FDBA958093490485
:105B900090934A04A0934B04B0934C042091920735
:105BA000309193074091940750919507809151044B
:105BB00090915204A0915304B0915404281B390BC6
:105BC0004A0B5B0B20939504309396044093970403
:105BD0005093980480916407E82EFF240027112732
:105BE000CA01B901A80197010E94C23CDA01C901AA
:105BF0002093A8043093A9044093AA045093AB04C3
:105C000057FF04C081509F4FAF4FBF4F892F9A2F2E
:105C1000AB2FBB27A7FDBA9590930A048093090484
:105C20008091960790919707A0919807B091990756
:105C300020914D0430914E0440914F0450915004F6
:105C4000821B930BA40BB50B8093990490939A0439
:105C5000A0939B04B0939C04BC01CD01A8019701C3
:105C60000E94C23CDA01C9012093AC043093AD0418
:105C70004093AE045093AF0457FF04C081509F4F30
:105C8000AF4FBF4FA92EBA2ECB2EDD24C7FCDA941E
:105C9000B0920C04A0920B0480918A0790918B071C
:105CA000A0918C07B0918D07B7FF04C081509F4F22
:105CB000AF4FBF4F892F9A2FAB2FBB27A7FDBA95A8
:105CC00080938A0790938B07A0938C07B0938D07DE
:105CD0008091820790918307A0918407B0918507F6
:105CE000B7FF04C081509F4FAF4FBF4F892F9A2FEE
:105CF000AB2FBB27A7FDBA958093820790938307AC
:105D0000A0938407B0938507E0905D04F0905E0453
:105D100000915F041091600480916104909162048D
:105D2000A0916304B0916404E81AF90A0A0B1B0BF2
:105D3000E0928D04F0928E0400938F0410939004EF
:105D400020915504309156044091570450915804C5
:105D50008091590490915A04A0915B04B0915C0425
:105D6000281B390B4A0B5B0B209391043093920450
:105D70004093930450939404E0929504F092960417
:105D800000939704109398042093990430939A04F5
:105D900040939B0450939C0480913D0490913E0459
:105DA000A0913F04B09140048E199F09A00BB10B44
:105DB00080933D0490933E04A0933F04B09340042D
:105DC0008091350490913604A0913704B091380445
:105DD000821B930BA40BB50B809335049093360470
:105DE000A0933704B09338048091510490915204E9
:105DF000A0915304B0915404BC01CD012AE130E0DC
:105E000040E050E00E94C23C3093D3062093D2067B
:105E100080914D0490914E04A0914F04B091500494
:105E2000BC01CD012AE130E040E050E00E94C23CDC
:105E30003093D5062093D4068091950490919604D2
:105E40009093D7068093D6068091990490919A04F6
:105E50009093D9068093D8068091920790919307EA
:105E6000A0919407B0919507BC01CD012AE130E0E3
:105E700040E050E00E94C23C3093DB062093DA06FB
:105E80008091960790919707A0919807B0919907F4
:105E9000BC01CD012AE130E040E050E00E94C23C6C
:105EA0003093DD062093DC068091AC049091AD0424
:105EB0009093EB068093EA06C50143E0880F991F93
:105EC0004A95E1F78A0D9B1D8A0D9B1D9093ED0667
:105ED0008093EC0681E090E09093B1048093B0044D
:105EE0002091B6043091B7044091B8045091B904A0
:105EF0008091920790919307A0919407B091950794
:105F0000281B390B4A0B5B0B57FF07C05095409578
:105F1000309521953F4F4F4F5F4F20523E444040B8
:105F200050400CF0FEC091E0E91690E1F90690E0D7
:105F3000090790E019070CF46CC08091B204882323
:105F400009F463C0D801C70117FF07C08827992744
:105F5000DC018E199F09A00BB10BB7FF04C0815063
:105F6000904FAF4FBF4F3CE0B595A795979587955C
:105F70003A95D1F701969093B1048093B004D8017B
:105F8000C70117FF03C00796A11DB11D23E0B595FA
:105F9000A795979587952A95D1F78093A804909314
:105FA000A904A093AA04B093AB0489589341A040DC
:105FB000B04064F088E893E1A0E0B0E08093A804EA
:105FC0009093A904A093AA04B093AB042091A804D1
:105FD0003091A9044091AA045091AB0457FF04C02A
:105FE00021503F4F4F4F5F4F232F342F452F5527C1
:105FF00047FD5A958091090490910A04820F931FDE
:1060000090930A048093090406C081E08093B2044F
:1060100002C01092B204E0909504F09096040091B2
:10602000970410919804F0E0EF16F0EFFF06FFEFF1
:106030000F07FFEF1F070CF071C08091B304882396
:1060400009F468C0A801970117FF07C0222733276A
:10605000A9012E193F09400B510B57FF04C02150D5
:10606000304F4F4F5F4F8CE05595479537952795AB
:106070008A95D1F78091B0049091B104820F931F5B
:106080009093B1048093B004D801C70117FF03C0F7
:106090000796A11DB11D13E0B595A7959795879516
:1060A0001A95D1F78093A8049093A904A093AA0409
:1060B000B093AB0488579C4EAF4FBF4F64F488E752
:1060C0009CEEAFEFBFEF8093A8049093A904A09338
:1060D000AA04B093AB042091A8043091A904409184
:1060E000AA045091AB0457FF04C021503F4F4F4FBB
:1060F0005F4F232F342F452F552747FD5A95809109
:10610000090490910A04820F931F90930A048093CC
:1061100009040BC081E08093B30407C01092B3045C
:1061200004C01092B1041092B00410916507212FA1
:1061300033278091B0049091B1042817390724F4D3
:106140003093B1042093B00440919504509196048B
:106150006091970470919804413034E0530730E027
:10616000630730E0730774F08091770490917804AE
:106170002091B0043091B104820F931F9093780462
:106180008093770440505C4F6F4F7F4F74F4809141
:106190007704909178042091B0043091B104821B6F
:1061A000930B909378048093770481E090E0909330
:1061B000B1048093B0041092AC041092AD0410921C
:1061C000AE041092AF042091BA043091BB04409108
:1061D000BC045091BD048091960790919707A091BF
:1061E0009807B0919907281B390B4A0B5B0B57FF97
:1061F00007C050954095309521953F4F4F4F5F4FC9
:1062000020523E44404050400CF000C1C0909904E0
:10621000D0909A04E0909B04F0909C04A1E0CA16F0
:10622000A0E1DA06A0E0EA06A0E0FA060CF46CC0F1
:106230008091B404882309F463C0D701C601F7FE36
:1062400007C088279927DC018C199D09AE09BF0971
:10625000B7FF04C08150904FAF4FBF4FFCE0B595E2
:10626000A79597958795FA95D1F701969093B104E4
:106270008093B004D701C601F7FE03C00796A11DA5
:10628000B11DE3E0B595A79597958795EA95D1F768
:106290008093AC049093AD04A093AE04B093AF048C
:1062A00089589341A040B04064F088E893E1A0E0B1
:1062B000B0E08093AC049093AD04A093AE04B0938F
:1062C000AF042091AC043091AD044091AE045091E4
:1062D000AF0457FF04C021503F4F4F4F5F4F232F54
:1062E000342F452F552747FD5A9580910B049091E7
:1062F0000C04820F931F90930C0480930B0406C030
:1063000081E08093B40402C01092B404F0E0CF1690
:10631000F0EFDF06FFEFEF06FFEFFF060CF073C0B4
:106320008091B504882309F46AC0D701C601F7FE3D
:1063300007C088279927DC018C199D09AE09BF0980
:106340009C01AD01B7FF04C02150304F4F4F5F4F4C
:106350006CE055954795379527956A95D1F78091CB
:10636000B0049091B104820F931F9093B104809375
:10637000B004D701C601F7FE03C00796A11DB11DE9
:1063800023E0B595A795979587952A95D1F78093A2
:10639000AC049093AD04A093AE04B093AF048857BF
:1063A0009C4EAF4FBF4F64F488E79CEEAFEFBFEF5A
:1063B0008093AC049093AD04A093AE04B093AF046B
:1063C0002091AC043091AD044091AE045091AF04E3
:1063D00057FF04C021503F4F4F4F5F4F232F342FA3
:1063E000452F552747FD5A9580910B0490910C0439
:1063F000820F931F90930C0480930B040BC081E0D9
:106400008093B50407C01092B50404C01092B10483
:106410001092B0048091AC049091AD049093E70683
:106420008093E606212F33278091B0049091B10428
:106430002817390724F43093B1042093B004409115
:10644000990450919A0460919B0470919C0441308E
:1064500034E0530730E0630730E0730774F0809155
:106460007504909176042091B0043091B104820FAC
:10647000931F909376048093750440505C4F6F4F48
:106480007F4F74F480917504909176042091B0044C
:106490003091B104821B930B909376048093750422
:1064A00080917704909178049093DF068093DE06C4
:1064B000209175043091760480917104909172045A
:1064C000281B390BC901B3E0880F991FBA95E1F772
:1064D000820F931F820F931F9093E1068093E00633
:1064E00008C010920C0410920B0410920A0410922F
:1064F000090480919A0790919B07A0919C07B09105
:106500009D0720E030E040E050E0BC01CD010E945A
:10651000963B882341F410920C0410920B041092C5
:106520000A04109209048091920790919307A09118
:106530009407B09195078093B6049093B704A09305
:10654000B804B093B9048091960790919707A091F1
:106550009807B09199078093BA049093BB04A093D5
:10656000BC04B093BD0410925104109252041092D6
:1065700053041092540410924D0410924E04109241
:106580004F04109250041092490410924A04109241
:106590004B0410924C0410929207109293071092A1
:1065A00094071092950710929607109297071092F1
:1065B00098071092990710928A0710928B071092F1
:1065C0008C0710928D071092820710928307109209
:1065D0008407109285071092CA031092C903A090F5
:1065E0001204B0901304C501B7FE04C08827992790
:1065F0008A199B0945973CF080913F0784FD03C0B1
:1066000081E08093A704D0904807ED2CFF24002759
:106610001127B501882777FD8095982F9501B7FE42
:1066200004C0222733272A193B09442737FD409508
:10663000542F0E944E3C9B01AC01C801B7010E943F
:106640004E3C97FF04C061507E4F8F4F9F4FA9E093
:106650009595879577956795AA95D1F79B018D2D8F
:1066600099278A9DD0018B9DB00D9A9DB00D112464
:10667000CD01B7FD03969595879595958795280F3C
:10668000391FC901AA2797FDA095BA2F80938904C5
:1066900090938A04A0938B04B0938C0420913104CE
:1066A000309132044091330450913404281B390B4B
:1066B0004A0B5B0B20933104309332044093330434
:1066C000509334048091310490913204A0913304AA
:1066D000B09134048155934CA040B04064F080E503
:1066E00093ECA0E0B0E08093310490933204A09347
:1066F0003304B09334048091310490913204A0911A
:106700003304B0913404805B9C43AF4FBF4F64F4BB
:1067100080EB9CE3AFEFBFEF8093310490933204A2
:10672000A0933304B09334048091270490912804FB
:10673000892B09F4AAC080913F0783FFA6C08091EE
:10674000610490916204A0916304B0916404B7FF66
:1067500004C081509E4FAF4FBF4FE9E0B595A7955C
:1067600097958795EA95D1F79C0197FF03C03095DF
:1067700021953F4F8091590490915A04A0915B0458
:10678000B0915C04B7FF04C081509E4FAF4FBF4F24
:1067900079E0B595A795979587957A95D1F7BC013E
:1067A00097FF03C0709561957F4F261737070CF44C
:1067B0009B0129313105A4F48091A704882381F03D
:1067C0008091BE049091BF04892B51F480912704DD
:1067D0009091280490932604809325041092A70496
:1067E00080917503482F5527249FC001259F900D48
:1067F000349F900D112497FDCF969C0166E035954E
:1068000027956A95E1F7421B530B9A01141615065A
:10681000B4F58091BE049091BF04009771F580910A
:10682000230490912404829FA001839F500D929F86
:10683000500D11249A0157FF02C0215E3F4F45E0E1
:10684000359527954A95E1F7442737FD4095542F14
:106850008091310490913204A0913304B0913404BA
:10686000820F931FA41FB51F8093310490933204AD
:10687000A0933304B093340408C0019702C084EF9E
:1068800091E09093BF048093BE048091A604815050
:106890008093A6048F3F09F085C088E18093A60409
:1068A00080914B07E82EFF24002711278091610477
:1068B00090916204A0916304B0916404BC01CD0185
:1068C000A80197010E94C23C3093B1062093B00604
:1068D0008091590490915A04A0915B04B0915C049A
:1068E000BC01CD01A80197010E94C23C3093B306C0
:1068F0002093B2068091A3079091A4079093B506C8
:106900008093B4068091AD079091AE079093B7063F
:106910008093B6068091A6079091A7079093B90639
:106920008093B80680910F04909110049093BB0659
:106930008093BA068091290490912A04A0912B0497
:10694000B0912C04B7FF04C081509E4FAF4FBF4F92
:1069500029E0B595A795979587952A95D1F79093B6
:10696000BD068093BC0680912704909128049093E3
:10697000C1068093C00680910E0390910F039093FF
:10698000C3068093C2068091180499279093C50688
:106990008093C40680918E0790918F079093D106C3
:1069A0008093D00680910804A090A807B090A90712
:1069B000C090AA07D090AB078823A9F080918707E1
:1069C00090918807AA2797FDA095BA2FBC01CD0109
:1069D0000E948C3BDC01CB01A6019501BC01CD01DD
:1069E0000E94063C3AC08091610490916204A0919B
:1069F0006304B0916404BC01CD010E948C3B7B0117
:106A00008C0180919A0790919B07A0919C07B0916F
:106A10009D079C01AD01C801B7010E94063C7B01A6
:106A20008C018091870790918807AA2797FDA095F0
:106A3000BA2FBC01CD010E948C3BDC01CB01A60129
:106A40009501BC01CD010E94063CDC01CB019C01FB
:106A5000AD01C801B7010E94E73ADC01CB01BC01DE
:106A6000CD010E946F3BDC01CB019093880780939E
:106A7000870780910704A090A807B090A907C0904D
:106A8000AA07D090AB078823A9F080917F07909147
:106A90008007AA2797FDA095BA2FBC01CD010E94BF
:106AA0008C3BDC01CB01A6019501BC01CD010E940C
:106AB000063C3AC08091590490915A04A0915B041D
:106AC000B0915C04BC01CD010E948C3B7B018C0128
:106AD00080919A0790919B07A0919C07B0919D0788
:106AE0009C01AD01C801B7010E94063C7B018C01ED
:106AF00080917F0790918007AA2797FDA095BA2FD4
:106B0000BC01CD010E948C3BDC01CB01A6019501AB
:106B1000BC01CD010E94063CDC01CB019C01AD0112
:106B2000C801B7010E94E73ADC01CB01BC01CD01ED
:106B30000E946F3BDC01CB019093800780937F071D
:106B40008091A6079091A707AA2797FDA095BA2F35
:106B5000BC01CD010E948C3B7B018C018091A80778
:106B60009091A907A091AA07B091AB079C01AD0134
:106B7000C801B7010E94063C7B018C01809145044D
:106B800090914604A0914704B0914804BC01CD0106
:106B90000E948C3BDC01CB0120909A0730909B0730
:106BA00040909C0750909D07A2019101BC01CD012E
:106BB0000E94063CDC01CB0120E030E040E05FE3D6
:106BC000BC01CD010E94063CDC01CB019C01AD0162
:106BD000C801B7010E94E73ADC01CB01BC01CD013D
:106BE0000E946F3BDC01CB019093A7078093A6071F
:106BF00080917F07909180079093E9068093E80643
:106C00008091590490915A04A0915B04B0915C0466
:106C1000BC01CD010E948C3BDC01CB01A2019101A2
:106C2000BC01CD010E94063CDC01CB01BC01CD01C1
:106C30000E946F3BDC01CB019093E3068093E20658
:106C400060911404709115047A8369837093EF0640
:106C50006093EE0680918707909188078150984055
:106C600034F080E098E090938807809387078091C4
:106C70008707909188078050984F34F480E098EF10
:106C8000909388078093870780917F079091800772
:106C90008150984034F080E098E090938007809392
:106CA0007F0780917F07909180078050984F34F440
:106CB00080E098EF9093800780937F078091A607EC
:106CC0009091A7078150984034F080E098E090932D
:106CD000A7078093A6078091A6079091A7078050E9
:106CE000984F34F480E098EF9093A7078093A6071D
:106CF00080913F07992780FFF1C02091780381FFA1
:106D00000EC0223310F580910F0490911004449727
:106D100090930E0480930D041092210419C0809169
:106D20006C0390916D03820F911D209144073327CE
:106D3000829FA001839F500D929F500D1124CA0184
:106D4000449790930E0480930D0481E08093210476
:106D5000992021F010920E0410920D0400910F045E
:106D60001091100420910D0430910E04201731076A
:106D70000CF0B4C080912104882309F4AFC0021B39
:106D8000130B809177039927089FB001099F700D1D
:106D9000189F700D1124CB0177FD0F968C0184E0B4
:106DA000159507958A95E1F7C301801B910B8C011E
:106DB00080917903282F33278091CB039091CC03C6
:106DC000829FD001839FB00D929FB00D1124CD0101
:106DD000B7FD0796B3E095958795BA95E1F7081B3F
:106DE000190BC0902904D0902A04E0902B04F09055
:106DF0002C04F7FE08C02FEF31E040E050E0C20E57
:106E0000D31EE41EF51EA9E0F594E794D794C79429
:106E1000AA95D1F780917603282F33274427552749
:106E2000C701B6010E944E3C97FF04C0615E7F4FD0
:106E30008F4F9F4FF5E09595879577956795FA95D4
:106E4000D1F7633371051CF062E370E006C03FEFD9
:106E50006E3C730714F46EEC7FEF061B170B8091EA
:106E6000A4049091A5049C01E4E0220F331FEA954D
:106E7000E1F7281B390B200F311F37FF02C0215FBC
:106E80003F4F74E0359527957A95E1F73093A50447
:106E90002093A40480914007482F552724173507D5
:106EA00074F46416750624F05093A5044093A4046A
:106EB0006416750624F47092A5046092A40480916F
:106EC000A4049091A5046816790624F47092A50490
:106ED0006092A4046090A4047090A5047092BF0610
:106EE0006092BE068090A6079090A70780918904C3
:106EF00090918A04881A990AC30177FC01969595A6
:106F00008795881599050CF44C01909581959F4FB4
:106F1000881699060CF44C014091A5074B83842FE9
:106F200099278619970997FD019695958795881554
:106F300099050CF44C01909581959F4F8816990600
:106F40000CF44C0154E16516710414F4882499245E
:106F500060911604709117048091D2049091D3042B
:106F6000681B790B7B876A878091870790918807D8
:106F7000861B970B909391078093900720E030E059
:106F800040E050E0C201B1010E94963B2091810493
:106F9000309182044091830450918404882309F441
:106FA00048C0CA01B9010E948C3B5B016C01809111
:106FB000610490916204A0916304B0916404BC01E7
:106FC000CD010E948C3BDC01CB01A2019101BC01EF
:106FD000CD010E94063C7B018C01EA85FB85CF0137
:106FE000AA2797FDA095BA2FBC01CD010E948C3B2A
:106FF000DC01CB019C01AD01C801B7010E94E63A5A
:10700000DC01CB019C01AD01C601B5010E94E73A4C
:10701000DC01CB01BC01CD010E946F3BDC01CB0147
:107020008093810490938204A0938304B09384049A
:1070300014C08091900790919107AA2797FDA09581
:10704000BA2F280F391F4A1F5B1F209381043093EA
:10705000820440938304509384048091810490912E
:107060008204A0918304B0918404181619061A06AC
:107070001B0624F40297A109B10903C00296A11DC1
:10708000B11D8093810490938204A0938304B093F4
:1070900084048091810490918204A0918304B09132
:1070A000840481589E43A040B04064F080E89EE391
:1070B000A0E0B0E08093810490938204A0938304C5
:1070C000B09384048091810490918204A091830400
:1070D000B09184048058914CAF4FBF4F64F480E866
:1070E00091ECAFEFBFEF8093810490938204A09363
:1070F0008304B09384048091900790919107AA270C
:1071000097FDA095BA2FBC01CD010E948C3B7B015D
:107110008C018091810490918204A0918304B091AC
:107120008404BC01CD010E948C3BDC01CB01409169
:107130007A0350917B0360917C0370917D034C83B3
:107140005D836E837F839C01AD016C817D818E8127
:107150009F810E94063CDC01CB019C01AD01C8016E
:10716000B7010E94E73ADC01CB01BC01CD010E94CE
:107170006F3BDC01CB018C0150916E035887652F6A
:10718000772788279927940197FE04C02227332761
:107190002819390937FF02C02F5F3F4F35952795D2
:1071A000260D371D442737FD4095542F0E944E3C35
:1071B00097FF04C0615C7F4F8F4F9F4FB6E095955E
:1071C000879577956795BA95D1F79B0160177107F9
:1071D0000CF48B0166277727621B730B06171707C2
:1071E0000CF48B019301200F311F280D391D37FF3F
:1071F00003C020E030E007C06B81862F99278217FB
:1072000093070CF49C01709189077987872F992740
:10721000281739070CF49C01209381079301201B48
:10722000310B280D391D37FF03C020E030E007C0C7
:107230008091A5079927821793070CF49C01A985D3
:107240008A2F9927281739070CF49C012093860769
:107250008091D0049091D104E981FA81E81BF90B67
:10726000FB87EA8780917F07909180078E1B9F0B99
:1072700090937E0780937D0720E030E040E050E06F
:10728000C201B1010E94963B209185043091860491
:107290004091870450918804882309F448C0CA01AA
:1072A000B9010E948C3B5B016C0180915904909163
:1072B0005A04A0915B04B0915C04BC01CD010E9412
:1072C0008C3BDC01CB01A2019101BC01CD010E94EC
:1072D000063C7B018C012A853B85C901AA2797FDC5
:1072E000A095BA2FBC01CD010E948C3BDC01CB01E3
:1072F0009C01AD01C801B7010E94E63ADC01CB0157
:107300009C01AD01C601B5010E94E73ADC01CB0149
:10731000BC01CD010E946F3BDC01CB018093850451
:1073200090938604A0938704B093880414C080913E
:107330007D0790917E07AA2797FDA095BA2F280F69
:10734000391F4A1F5B1F20938504309386044093A6
:107350008704509388048091850490918604A091BD
:107360008704B0918804181619061A061B0624F41F
:107370000297A109B10903C00296A11DB11D809316
:10738000850490938604A0938704B0938804809129
:10739000850490918604A0918704B0918804815857
:1073A0009E43A040B04064F080E89EE3A0E0B0E0DF
:1073B0008093850490938604A0938704B0938804F7
:1073C0008091850490918604A0918704B0918804EF
:1073D0008058914CAF4FBF4F64F480E891ECAFEF11
:1073E000BFEF8093850490938604A0938704B093A5
:1073F000880480917D0790917E07AA2797FDA0952C
:10740000BA2FBC01CD010E948C3B7B018C01809185
:10741000850490918604A0918704B0918804BC01F2
:10742000CD010E948C3BDC01CB019C01AD016C8144
:107430007D818E819F810E94063CDC01CB019C01F5
:10744000AD01C801B7010E94E73ADC01CB01BC01E4
:10745000CD010E946F3BDC01CB018C015885652F6B
:10746000772788279927940197FE04C0222733277E
:107470002819390937FF02C02F5F3F4F35952795EF
:10748000260D371D442737FD4095542F0E944E3C52
:1074900097FF04C0615C7F4F8F4F9F4FF6E095953B
:1074A000879577956795FA95D1F79B0160177107D6
:1074B0000CF48B0166277727621B730B06171707DF
:1074C0000CF48B019301200F311F2819390937FF64
:1074D00003C020E030E007C08091A50799278217FC
:1074E00093070CF49C016985862F99272817390783
:1074F0000CF49C012093A0079301201B310B281949
:10750000390937FF03C020E030E007C08091A507AC
:107510009927821793070CF49C017985872F992767
:10752000281739070CF49C0120939E072B960FB661
:10753000F894DEBF0FBECDBFDF91CF911F910F91A9
:10754000FF90EF90DF90CF90BF90AF909F908F9083
:107550007F906F905F904F903F902F900895809113
:10756000CC049091CD04A091CE04B091CF0480932F
:10757000C4049093C504A093C604B093C70480913B
:10758000C8049091C904A091CA04B091CB0480931F
:10759000C0049093C104A093C204B093C30408959F
:1075A0001092D3041092D2041092D1041092D004FD
:1075B0000895FC014150504030F001900616D1F77B
:1075C0003197CF0108958827992708955058192E8B
:1075D000EFD001D0D2C0BA176207730784079507AE
:1075E000B1F188F40EF410940B2EBA2FA02D062EB4
:1075F000622F202D072E732F302D082E842F402D23
:10760000092E952F502DFF275523B9F0591B49F00E
:10761000573E98F0469537952795A795F040539596
:10762000C9F776F0BA0F621F731F841F30F4879575
:1076300077956795B795F040939517FA0F2E0895B3
:10764000BF1BBB27BA0B620B730B840BF6CFDEF6A6
:10765000DBC0AED001D091C0552359F0992369F019
:107660009F575F57951B33F442F4903811F49158AB
:1076700005C09BC091589F3F09F4C6C0BB27112489
:1076800062177307840730F4660F771F881FBB1FCC
:10769000915098F311D00F920FD00F920DD0A0E817
:1076A0002617370748071B0609F0A048BA2F602D98
:1076B0007F918F9100240895A0E80024621773073A
:1076C0008407B10528F0621B730B840BB1090A2AE9
:1076D000660F771F881FBB1FA69581F7089597FB3C
:1076E00073D09F3738F0FEE9F91B982F872F762F3C
:1076F0006B2F05C086C09695879577956795F15055
:10770000D0F73EF490958095709561957F4F8F4F9F
:107710009F4F0895E89403C097FB0EF4F3DFB62F54
:10772000672F782F892F9EE9002427C00ED05EF0A6
:1077300004C00BD026F001C008D019F020F48FEF60
:10774000089580E0089581E0089597FB092E0526AD
:1077500000F8689430D0E89407FC07C062177307FC
:107760008407950721F008F40094079498940895ED
:107770009A95BB0F661F771F881F11249923A1F0CC
:107780008823B2F79F3F59F0BB0F48F421F4002043
:1077900011F460FF04C06F5F7F4F8F4F9F4F881FB2
:1077A0009795879597F908952CC09FEF80EC0895E1
:1077B000052E092607FA440F551F5F3F79F0AA27C7
:1077C000A51708F051E04795880F991F9F3F31F0AA
:1077D000BB27B91708F091E0879508959F919F9175
:1077E0001124E3CF97FB880F991F9F3F31F0BB27F0
:1077F000B91708F091E0879508959F919F91112402
:10780000D4CF66277727882799270895D1DF01D01D
:10781000B4CF992339F0552329F09F575F57950F1F
:1078200013F49AF1F1CF91589F3FE1F3629FA12D9C
:107830000F92BB27639FA00DB11DEE27729FA00D75
:10784000B11DEE1FAF93AA27649FB00DE11D739F7A
:10785000B00DE11DAA1F6627829FB00DE11DA61F76
:107860005527749FE00DA11D551F839FE00DA11D9D
:10787000561F849FA00D511D852F7A2F6E2F1F90AC
:107880000F9088231AF4939539F48FCF000C111CB4
:10789000BB1F661F771F881F01280895629FD001B4
:1078A000739FF001829FE00DF11D649FE00DF11DBB
:1078B000929FF00D839FF00D749FF00D659FF00D6A
:1078C0009927729FB00DE11DF91F639FB00DE11D57
:1078D000F91FBD01CF0111240895991B79E004C05F
:1078E000991F961708F0961B881F7A95C9F78095FF
:1078F0000895AA1BBB1B51E107C0AA1FBB1FA617F7
:10790000B70710F0A61BB70B881F991F5A95A9F748
:1079100080959095BC01CD01089597FB092E07260F
:107920000AD077FD04D0E5DF06D000201AF4709568
:1079300061957F4F0895F6F7909581959F4F089533
:10794000A1E21A2EAA1BBB1BFD010DC0AA1FBB1F63
:10795000EE1FFF1FA217B307E407F50720F0A21BD5
:10796000B30BE40BF50B661F771F881F991F1A9442
:1079700069F760957095809590959B01AC01BD016C
:10798000CF01089597FB092E05260ED057FD04D090
:10799000D7DF0AD0001C38F45095409530952195DA
:1079A0003F4F4F4F5F4F0895F6F790958095709534
:1079B00061957F4F8F4F9F4F0895F999FECFB2BDCC
:1079C000A1BDF89A119600B40895F999FECFB2BD01
:1079D000A1BD00BC11960FB6F894FA9AF99A0FBEA1
:0279E000089508
:1079E2000A496E74656772616C4E69636B20202070
:1079F20020496E74656772616C526F6C6C20202036
:107A0200204163634E69636B2020202020202020C8
:107A120020416363526F6C6C2020202020202020A4
:107A2200204779726F47696572202020202020202C
:107A320020486F6568656E5765727420202020208B
:107A4200204163635A202020202020202020202053
:107A52002047617320202020202020202020202069
:107A6200204B6F6D7061737356616C7565202020B9
:107A7200205370616E6E756E6720202020202020BA
:107A820020456D7066616E67202020202020202016
:107A9200203131202D2D2D2020202020202020209B
:107AA200204D6F746F725F566F726E6520202020BA
:107AB200204D6F746F725F48696E74656E2020206E
:107AC200204D6F746F725F4C696E6B7320202020A3
:107AD200204D6F746F725F5265636874732020204B
:107AE2002031365F4163635F5A202020202020200E
:107AF2002031374D697474656C4163634E69636B01
:107B02002031385F4D697474656C416363526F6CE8
:107B12006C416E616C6F673139202020202020205B
:107B220020496E74656772616C457272526F6C6C3B
:107B320020416E616C6F673231202020202020208E
:107B42002032325F4D697474656C47496E6752200A
:107B520020416E616C6F673233202020202020206C
:107B6200203234526F6C6C4F66667365742020202D
:107B7200203235496E74526F6C6C2A46616B7420E8
:107B820020416E616C6F6732362020202020202039
:107B920020446972656B74417573676C526F6C6CCB
:107BA2002032384D65737377657274526F6C6C2036
:107BB200203239417573676C65696368526F6C6C0A
:107BC2002033305F492D4C616765526F6C6C202009
:107BD2002033315F537469636B526F6C6C202020C9
:107BE2002064FF01FFFF010AFF03007D0000640023
:107BF20048616C6C6F2057656C74000000000000D7
:107C02000000000000000000000000000000000072
:107C12000000000000000000000000000000000062
:107C22000000000000000000000000000000000052
:107C32000000000000000000000000000000000042
:107C42000102030405060708090A0A01ECFF64465B
:107C5200640A029696403A10FB3017B7D13890D09A
:107C6200030090D00300640053706F727400004EE2
:107C72006F726D616C0000426567696E6E657200BD
:027C8200000000
:00000001FF
